 flexcan

 Timestamp is 4fb05c7c (Mon May 14 13:14:36 2012)

 Preferred load address is 10000000

 Start         Length     Name                   Class
 0001:00000000 00000004H .CRT$XCA                CODE
 0001:00000004 00000004H .CRT$XCZ                CODE
 0001:00000008 00000004H .CRT$XIA                CODE
 0001:0000000c 00000004H .CRT$XIZ                CODE
 0001:00000010 00000004H .CRT$XPA                CODE
 0001:00000014 00000004H .CRT$XPZ                CODE
 0001:00000018 00000004H .CRT$XTA                CODE
 0001:0000001c 00000004H .CRT$XTZ                CODE
 0001:00000020 00005b94H .rdata                  CODE
 0001:00005bb4 00000024H .rdata$debug            CODE
 0001:00005bd8 00008a18H .text                   CODE
 0001:0000e5f0 0000002cH .xdata                  CODE
 0001:0000e61c 0000003cH .idata$2                CODE
 0001:0000e658 00000014H .idata$3                CODE
 0001:0000e66c 000000ecH .idata$4                CODE
 0001:0000e758 000000a6H .idata$6                CODE
 0001:0000e800 000000b5H .edata                  CODE
 0002:00000000 000000ecH .idata$5                DATA
 0002:000000f0 0000044cH .data                   DATA
 0002:00000540 00000fb8H .bss                    DATA
 0003:00000000 000002d8H .pdata                  DATA

  Address         Publics by Value              Rva+Base       Lib:Object

 0000:00000000       ___safe_se_handler_table   00000000     <absolute>
 0000:00000000       ___safe_se_handler_count   00000000     <absolute>
 0001:00000000       __xc_a                     10001000     corelib0:crt0init.obj
 0001:00000004       __xc_z                     10001004     corelib0:crt0init.obj
 0001:00000008       __xi_a                     10001008     corelib0:crt0init.obj
 0001:0000000c       __xi_z                     1000100c     corelib0:crt0init.obj
 0001:00000010       __xp_a                     10001010     corelib0:crt0init.obj
 0001:00000014       __xp_z                     10001014     corelib0:crt0init.obj
 0001:00000018       __xt_a                     10001018     corelib0:crt0init.obj
 0001:0000001c       __xt_z                     1000101c     corelib0:crt0init.obj
 0001:00000040       ??_C@_1EE@JBEAFIDI@?$AAF?$AAl?$AAe?$AAx?$AAC?$AAA?$AAN?$AA?5?$AAD?$AAr?$AAi?$AAv?$AAe?$AAr?$AA?3?$AA?5?$AA?9?$AAD?$AAl?$AAl?$AAM?$AAa?$AAi?$AAn?$AA?$CI?$AAT?$AAR?$AAU?$AAE?$AA?$CJ?$AA?9?$AA?$AN@ 10001040     driver.obj
 0001:00000088       ??_C@_1IG@MHDADDNM@?$AAF?$AAl?$AAe?$AAx?$AAC?$AAA?$AAN?$AA?5?$AAD?$AAr?$AAi?$AAv?$AAe?$AAr?$AA?3?$AA?5?$AA?$CL?$AAD?$AAl?$AAl?$AAM?$AAa?$AAi?$AAn?$AA?$CI?$AAh?$AAI?$AAn?$AAs?$AAt?$AAa?$AAn@ 10001088     driver.obj
 0001:00000110       ??_C@_1EC@CGAALHJA@?$AAF?$AAl?$AAe?$AAx?$AAC?$AAA?$AAN?$AA?5?$AAD?$AAr?$AAi?$AAv?$AAe?$AAr?$AA?3?$AA?5?$AA?9?$AAI?$AAn?$AAi?$AAt?$AA?$CI?$AA0?$AAx?$AA?$CF?$AA0?$AA8?$AAX?$AA?$CJ?$AA?9?$AA?$AN?$AA?6@ 10001110     driver.obj
 0001:00000158       ??_C@_1IM@CFPLDPKP@?$AAF?$AAl?$AAe?$AAx?$AAC?$AAA?$AAN?$AA?5?$AAD?$AAr?$AAi?$AAv?$AAe?$AAr?$AA?3?$AA?5?$AA?5?$AAI?$AAn?$AAi?$AAt?$AA?$DO?$AA?5?$AAE?$AAR?$AAR?$AAO?$AAR?$AA?3?$AA?5?$AAE?$AAr@ 10001158     driver.obj
 0001:000001e8       ??_C@_1HG@PGOFFHCM@?$AAF?$AAl?$AAe?$AAx?$AAC?$AAA?$AAN?$AA?5?$AAD?$AAr?$AAi?$AAv?$AAe?$AAr?$AA?3?$AA?5?$AA?5?$AAI?$AAn?$AAi?$AAt?$AA?$DO?$AA?5?$AAE?$AAR?$AAR?$AAO?$AAR?$AA?3?$AA?5?$AAE?$AAr@ 100011e8     driver.obj
 0001:00000260       ??_C@_1GG@HHILMIEE@?$AAF?$AAl?$AAe?$AAx?$AAC?$AAA?$AAN?$AA?5?$AAD?$AAr?$AAi?$AAv?$AAe?$AAr?$AA?3?$AA?5?$AA?$CL?$AAI?$AAn?$AAi?$AAt?$AA?$CI?$AAp?$AAs?$AAz?$AAA?$AAc?$AAt?$AAi?$AAv?$AAe?$AAK@ 10001260     driver.obj
 0001:000002c8       ??_C@_1DO@JEJFPAKD@?$AAF?$AAl?$AAe?$AAx?$AAC?$AAA?$AAN?$AA?5?$AAD?$AAr?$AAi?$AAv?$AAe?$AAr?$AA?3?$AA?5?$AA?9?$AAD?$AAe?$AAi?$AAn?$AAi?$AAt?$AA?$CI?$AA?$CF?$AAs?$AA?$CJ?$AA?9?$AA?$AN?$AA?6?$AA?$AA@ 100012c8     driver.obj
 0001:00000308       ??_C@_1M@HCOOECOK@?$AAF?$AAA?$AAL?$AAS?$AAE?$AA?$AA@ 10001308     driver.obj
 0001:00000314       ??_C@_19ELAAHEEL@?$AAT?$AAR?$AAU?$AAE?$AA?$AA@ 10001314     driver.obj
 0001:00000320       ??_C@_1GC@OCKFLDCD@?$AAF?$AAl?$AAe?$AAx?$AAC?$AAA?$AAN?$AA?5?$AAD?$AAr?$AAi?$AAv?$AAe?$AAr?$AA?3?$AA?5?$AA?$CL?$AAD?$AAe?$AAi?$AAn?$AAi?$AAt?$AA?$CI?$AAp?$AAD?$AAr?$AAi?$AAv?$AAe?$AAr?$AAI@ 10001320     driver.obj
 0001:00000388       ??_C@_1EC@EPNOOJKL@?$AAF?$AAl?$AAe?$AAx?$AAC?$AAA?$AAN?$AA?5?$AAD?$AAr?$AAi?$AAv?$AAe?$AAr?$AA?3?$AA?5?$AA?9?$AAO?$AAp?$AAe?$AAn?$AA?$CI?$AA0?$AAx?$AA?$CF?$AA0?$AA8?$AAX?$AA?$CJ?$AA?9?$AA?$AN?$AA?6@ 10001388     driver.obj
 0001:000003d0       ??_C@_1FO@PKNDMMIK@?$AAF?$AAl?$AAe?$AAx?$AAC?$AAA?$AAN?$AA?5?$AAD?$AAr?$AAi?$AAv?$AAe?$AAr?$AA?3?$AA?5?$AA?5?$AAO?$AAp?$AAe?$AAn?$AA?$DO?$AA?5?$AAI?$AAN?$AAV?$AAA?$AAL?$AAI?$AAD?$AA_?$AAH@ 100013d0     driver.obj
 0001:00000430       ??_C@_1JM@DKEJCPCG@?$AAF?$AAl?$AAe?$AAx?$AAC?$AAA?$AAN?$AA?5?$AAD?$AAr?$AAi?$AAv?$AAe?$AAr?$AA?3?$AA?5?$AA?5?$AAO?$AAp?$AAe?$AAn?$AA?$DO?$AA?5?$AAE?$AAR?$AAR?$AAO?$AAR?$AA?3?$AA?5?$AAC?$AAa@ 10001430     driver.obj
 0001:000004d0       ??_C@_1FO@NFHJIEJL@?$AAF?$AAl?$AAe?$AAx?$AAC?$AAA?$AAN?$AA?5?$AAD?$AAr?$AAi?$AAv?$AAe?$AAr?$AA?3?$AA?5?$AA?$CL?$AAO?$AAp?$AAe?$AAn?$AA?$CI?$AAp?$AAD?$AAr?$AAi?$AAv?$AAe?$AAr?$AAI?$AAn?$AAf@ 100014d0     driver.obj
 0001:00000530       ??_C@_1EC@DDGLKGPD@?$AAF?$AAl?$AAe?$AAx?$AAC?$AAA?$AAN?$AA?5?$AAD?$AAr?$AAi?$AAv?$AAe?$AAr?$AA?3?$AA?5?$AA?9?$AAP?$AAr?$AAe?$AAC?$AAl?$AAo?$AAs?$AAe?$AA?$CI?$AA?$CF?$AAs?$AA?$CJ?$AA?9?$AA?$AN?$AA?6@ 10001530     driver.obj
 0001:00000578       ??_C@_1GC@EBFCEDCP@?$AAF?$AAl?$AAe?$AAx?$AAC?$AAA?$AAN?$AA?5?$AAD?$AAr?$AAi?$AAv?$AAe?$AAr?$AA?3?$AA?5?$AA?$CL?$AAP?$AAr?$AAe?$AAC?$AAl?$AAo?$AAs?$AAe?$AA?$CI?$AAp?$AAO?$AAp?$AAe?$AAn?$AAI@ 10001578     driver.obj
 0001:000005dc       ??_C@_1DM@ONJODOAJ@?$AAF?$AAl?$AAe?$AAx?$AAC?$AAA?$AAN?$AA?5?$AAD?$AAr?$AAi?$AAv?$AAe?$AAr?$AA?3?$AA?5?$AA?9?$AAC?$AAl?$AAo?$AAs?$AAe?$AA?$CI?$AA?$CF?$AAs?$AA?$CJ?$AA?9?$AA?$AN?$AA?6?$AA?$AA@ 100015dc     driver.obj
 0001:00000618       ??_C@_1GA@MIHEJDAP@?$AAF?$AAl?$AAe?$AAx?$AAC?$AAA?$AAN?$AA?5?$AAD?$AAr?$AAi?$AAv?$AAe?$AAr?$AA?3?$AA?5?$AA?5?$AAC?$AAl?$AAo?$AAs?$AAe?$AA?$DO?$AA?5?$AAI?$AAN?$AAV?$AAA?$AAL?$AAI?$AAD?$AA_@ 10001618     driver.obj
 0001:00000678       ??_C@_1FM@EOPKJAPF@?$AAF?$AAl?$AAe?$AAx?$AAC?$AAA?$AAN?$AA?5?$AAD?$AAr?$AAi?$AAv?$AAe?$AAr?$AA?3?$AA?5?$AA?$CL?$AAC?$AAl?$AAo?$AAs?$AAe?$AA?$CI?$AAp?$AAO?$AAp?$AAe?$AAn?$AAI?$AAn?$AAf?$AAo@ 10001678     driver.obj
 0001:000006d4       ??_C@_1DK@JDKJJLOI@?$AAF?$AAl?$AAe?$AAx?$AAC?$AAA?$AAN?$AA?5?$AAD?$AAr?$AAi?$AAv?$AAe?$AAr?$AA?3?$AA?5?$AA?9?$AAR?$AAe?$AAa?$AAd?$AA?$CI?$AA?$CF?$AAd?$AA?$CJ?$AA?9?$AA?$AN?$AA?6?$AA?$AA@ 100016d4     driver.obj
 0001:00000710       ??_C@_1FK@KEJLNKIK@?$AAF?$AAl?$AAe?$AAx?$AAC?$AAA?$AAN?$AA?5?$AAD?$AAr?$AAi?$AAv?$AAe?$AAr?$AA?3?$AA?5?$AA?$CL?$AAR?$AAe?$AAa?$AAd?$AA?$CI?$AAp?$AAO?$AAp?$AAe?$AAn?$AAI?$AAn?$AAf?$AAo?$AA?5@ 10001710     driver.obj
 0001:0000076c       ??_C@_1DM@JLDGBKBM@?$AAF?$AAl?$AAe?$AAx?$AAC?$AAA?$AAN?$AA?5?$AAD?$AAr?$AAi?$AAv?$AAe?$AAr?$AA?3?$AA?5?$AA?9?$AAW?$AAr?$AAi?$AAt?$AAe?$AA?$CI?$AA?$CF?$AAd?$AA?$CJ?$AA?9?$AA?$AN?$AA?6?$AA?$AA@ 1000176c     driver.obj
 0001:000007a8       ??_C@_1FM@KJPNIOOD@?$AAF?$AAl?$AAe?$AAx?$AAC?$AAA?$AAN?$AA?5?$AAD?$AAr?$AAi?$AAv?$AAe?$AAr?$AA?3?$AA?5?$AA?$CL?$AAW?$AAr?$AAi?$AAt?$AAe?$AA?$CI?$AAp?$AAO?$AAp?$AAe?$AAn?$AAI?$AAn?$AAf?$AAo@ 100017a8     driver.obj
 0001:00000804       ??_C@_1DK@DNJPICNE@?$AAF?$AAl?$AAe?$AAx?$AAC?$AAA?$AAN?$AA?5?$AAD?$AAr?$AAi?$AAv?$AAe?$AAr?$AA?3?$AA?5?$AA?9?$AAS?$AAe?$AAe?$AAk?$AA?$CI?$AA?9?$AA1?$AA?$CJ?$AA?9?$AA?$AN?$AA?6?$AA?$AA@ 10001804     driver.obj
 0001:00000840       ??_C@_1FO@FGLKJFHE@?$AAF?$AAl?$AAe?$AAx?$AAC?$AAA?$AAN?$AA?5?$AAD?$AAr?$AAi?$AAv?$AAe?$AAr?$AA?3?$AA?5?$AA?5?$AAS?$AAe?$AAe?$AAk?$AA?$DO?$AA?5?$AAI?$AAN?$AAV?$AAA?$AAL?$AAI?$AAD?$AA_?$AAH@ 10001840     driver.obj
 0001:000008a0       ??_C@_1FK@MDKGKFBM@?$AAF?$AAl?$AAe?$AAx?$AAC?$AAA?$AAN?$AA?5?$AAD?$AAr?$AAi?$AAv?$AAe?$AAr?$AA?3?$AA?5?$AA?5?$AAS?$AAe?$AAe?$AAk?$AA?$DO?$AA?5?$AAE?$AAR?$AAR?$AAO?$AAR?$AA_?$AAN?$AAO?$AAT@ 100018a0     driver.obj
 0001:00000900       ??_C@_1FK@BFJHKEHD@?$AAF?$AAl?$AAe?$AAx?$AAC?$AAA?$AAN?$AA?5?$AAD?$AAr?$AAi?$AAv?$AAe?$AAr?$AA?3?$AA?5?$AA?$CL?$AAS?$AAe?$AAe?$AAk?$AA?$CI?$AAp?$AAO?$AAp?$AAe?$AAn?$AAI?$AAn?$AAf?$AAo?$AA?5@ 10001900     driver.obj
 0001:00000960       ??_C@_1EE@HMEBPFPI@?$AAF?$AAl?$AAe?$AAx?$AAC?$AAA?$AAN?$AA?5?$AAD?$AAr?$AAi?$AAv?$AAe?$AAr?$AA?3?$AA?5?$AA?9?$AAI?$AAO?$AAC?$AAo?$AAn?$AAt?$AAr?$AAo?$AAl?$AA?$CI?$AA?$CF?$AAs?$AA?$CJ?$AA?9?$AA?$AN@ 10001960     driver.obj
 0001:000009a8       ??_C@_1GG@CNGNNDPP@?$AAF?$AAl?$AAe?$AAx?$AAC?$AAA?$AAN?$AA?5?$AAD?$AAr?$AAi?$AAv?$AAe?$AAr?$AA?3?$AA?5?$AA?5?$AAI?$AAO?$AAC?$AAo?$AAn?$AAt?$AAr?$AAo?$AAl?$AA?$DO?$AA?5?$AAE?$AAR?$AAR?$AAO@ 100019a8     driver.obj
 0001:00000a10       ??_C@_1GE@PKBABNED@?$AAF?$AAl?$AAe?$AAx?$AAC?$AAA?$AAN?$AA?5?$AAD?$AAr?$AAi?$AAv?$AAe?$AAr?$AA?3?$AA?5?$AA?5?$AAI?$AAO?$AAC?$AAo?$AAn?$AAt?$AAr?$AAo?$AAl?$AA?$DO?$AA?5?$AAE?$AAR?$AAR?$AAO@ 10001a10     driver.obj
 0001:00000a78       ??_C@_1FM@PEGBIJPG@?$AAF?$AAl?$AAe?$AAx?$AAC?$AAA?$AAN?$AA?5?$AAD?$AAr?$AAi?$AAv?$AAe?$AAr?$AA?3?$AA?5?$AA?5?$AAI?$AAO?$AAC?$AAo?$AAn?$AAt?$AAr?$AAo?$AAl?$AA?$DO?$AA?5?$AAI?$AAO?$AAC?$AAT@ 10001a78     driver.obj
 0001:00000ad8       ??_C@_1FM@PLHPFPHF@?$AAF?$AAl?$AAe?$AAx?$AAC?$AAA?$AAN?$AA?5?$AAD?$AAr?$AAi?$AAv?$AAe?$AAr?$AA?3?$AA?5?$AA?5?$AAI?$AAO?$AAC?$AAo?$AAn?$AAt?$AAr?$AAo?$AAl?$AA?$DO?$AA?5?$AAI?$AAO?$AAC?$AAT@ 10001ad8     driver.obj
 0001:00000b38       ??_C@_1GO@KPJANPDC@?$AAF?$AAl?$AAe?$AAx?$AAC?$AAA?$AAN?$AA?5?$AAD?$AAr?$AAi?$AAv?$AAe?$AAr?$AA?3?$AA?5?$AA?5?$AAI?$AAO?$AAC?$AAo?$AAn?$AAt?$AAr?$AAo?$AAl?$AA?$DO?$AA?5?$AAI?$AAO?$AAC?$AAT@ 10001b38     driver.obj
 0001:00000ba8       ??_C@_1GK@CFMINJON@?$AAF?$AAl?$AAe?$AAx?$AAC?$AAA?$AAN?$AA?5?$AAD?$AAr?$AAi?$AAv?$AAe?$AAr?$AA?3?$AA?5?$AA?5?$AAI?$AAO?$AAC?$AAo?$AAn?$AAt?$AAr?$AAo?$AAl?$AA?$DO?$AA?5?$AAI?$AAO?$AAC?$AAT@ 10001ba8     driver.obj
 0001:00000c18       ??_C@_1GI@FCFLMMAM@?$AAF?$AAl?$AAe?$AAx?$AAC?$AAA?$AAN?$AA?5?$AAD?$AAr?$AAi?$AAv?$AAe?$AAr?$AA?3?$AA?5?$AA?5?$AAI?$AAO?$AAC?$AAo?$AAn?$AAt?$AAr?$AAo?$AAl?$AA?$DO?$AA?5?$AAI?$AAO?$AAC?$AAT@ 10001c18     driver.obj
 0001:00000c80       ??_C@_1BBC@HMFOCHAB@?$AAF?$AAl?$AAe?$AAx?$AAC?$AAA?$AAN?$AA?5?$AAD?$AAr?$AAi?$AAv?$AAe?$AAr?$AA?3?$AA?5?$AA?$CL?$AAI?$AAO?$AAC?$AAo?$AAn?$AAt?$AAr?$AAo?$AAl?$AA?$CI?$AAp?$AAO?$AAp?$AAe?$AAn@ 10001c80     driver.obj
 0001:00000d94       ??_7?$Buffer_t@VDuplicateTraits_t@detail@marshal@ce@@@detail@marshal@ce@@6B@ 10001d94     driver.obj
 0001:00000d98       ?dwCANRegisterValues@FlexCAN@@0QBKB 10001d98     flexcan.obj
 0001:00000de0       ??_C@_1FI@BJBAJEHC@?$AAF?$AAl?$AAe?$AAx?$AAC?$AAA?$AAN?$AA?5?$AAD?$AAr?$AAi?$AAv?$AAe?$AAr?$AA?3?$AA?5?$AA?9?$AAF?$AAl?$AAe?$AAx?$AAC?$AAA?$AAN?$AA?3?$AA?3?$AAI?$AAn?$AAi?$AAt?$AAi?$AAa@ 10001de0     flexcan.obj
 0001:00000e38       ??_C@_1JI@EFPPOIDK@?$AAF?$AAl?$AAe?$AAx?$AAC?$AAA?$AAN?$AA?5?$AAD?$AAr?$AAi?$AAv?$AAe?$AAr?$AA?3?$AA?5?$AA?5?$AAF?$AAl?$AAe?$AAx?$AAC?$AAA?$AAN?$AA?3?$AA?3?$AAI?$AAn?$AAi?$AAt?$AAi?$AAa@ 10001e38     flexcan.obj
 0001:00000ed0       ??_C@_1NA@GFLDNAGJ@?$AAF?$AAl?$AAe?$AAx?$AAC?$AAA?$AAN?$AA?5?$AAD?$AAr?$AAi?$AAv?$AAe?$AAr?$AA?3?$AA?5?$AA?5?$AAF?$AAl?$AAe?$AAx?$AAC?$AAA?$AAN?$AA?3?$AA?3?$AAI?$AAn?$AAi?$AAt?$AAi?$AAa@ 10001ed0     flexcan.obj
 0001:00000fa0       ??_C@_1LO@KBPJCALD@?$AAF?$AAl?$AAe?$AAx?$AAC?$AAA?$AAN?$AA?5?$AAD?$AAr?$AAi?$AAv?$AAe?$AAr?$AA?3?$AA?5?$AA?5?$AAF?$AAl?$AAe?$AAx?$AAC?$AAA?$AAN?$AA?3?$AA?3?$AAI?$AAn?$AAi?$AAt?$AAi?$AAa@ 10001fa0     flexcan.obj
 0001:00001060       ??_C@_1LK@DCLIMOGP@?$AAF?$AAl?$AAe?$AAx?$AAC?$AAA?$AAN?$AA?5?$AAD?$AAr?$AAi?$AAv?$AAe?$AAr?$AA?3?$AA?5?$AA?5?$AAF?$AAl?$AAe?$AAx?$AAC?$AAA?$AAN?$AA?3?$AA?3?$AAI?$AAn?$AAi?$AAt?$AAi?$AAa@ 10002060     flexcan.obj
 0001:00001120       ??_C@_1LO@HPBKMJFD@?$AAF?$AAl?$AAe?$AAx?$AAC?$AAA?$AAN?$AA?5?$AAD?$AAr?$AAi?$AAv?$AAe?$AAr?$AA?3?$AA?5?$AA?5?$AAF?$AAl?$AAe?$AAx?$AAC?$AAA?$AAN?$AA?3?$AA?3?$AAI?$AAn?$AAi?$AAt?$AAi?$AAa@ 10002120     flexcan.obj
 0001:000011e0       ??_C@_1NI@KHJPCICC@?$AAF?$AAl?$AAe?$AAx?$AAC?$AAA?$AAN?$AA?5?$AAD?$AAr?$AAi?$AAv?$AAe?$AAr?$AA?3?$AA?5?$AA?5?$AAF?$AAl?$AAe?$AAx?$AAC?$AAA?$AAN?$AA?3?$AA?3?$AAI?$AAn?$AAi?$AAt?$AAi?$AAa@ 100021e0     flexcan.obj
 0001:000012b8       ??_C@_1LI@PCKCLCBH@?$AAF?$AAl?$AAe?$AAx?$AAC?$AAA?$AAN?$AA?5?$AAD?$AAr?$AAi?$AAv?$AAe?$AAr?$AA?3?$AA?5?$AA?5?$AAF?$AAl?$AAe?$AAx?$AAC?$AAA?$AAN?$AA?3?$AA?3?$AAI?$AAn?$AAi?$AAt?$AAi?$AAa@ 100022b8     flexcan.obj
 0001:00001370       ??_C@_1JA@EKJFDDME@?$AAF?$AAl?$AAe?$AAx?$AAC?$AAA?$AAN?$AA?5?$AAD?$AAr?$AAi?$AAv?$AAe?$AAr?$AA?3?$AA?5?$AA?5?$AAF?$AAl?$AAe?$AAx?$AAC?$AAA?$AAN?$AA?3?$AA?3?$AAI?$AAn?$AAi?$AAt?$AAi?$AAa@ 10002370     flexcan.obj
 0001:00001400       ??_C@_1HK@BLBFNKEL@?$AAF?$AAl?$AAe?$AAx?$AAC?$AAA?$AAN?$AA?5?$AAD?$AAr?$AAi?$AAv?$AAe?$AAr?$AA?3?$AA?5?$AA?$CL?$AAF?$AAl?$AAe?$AAx?$AAC?$AAA?$AAN?$AA?3?$AA?3?$AAI?$AAn?$AAi?$AAt?$AAi?$AAa@ 10002400     flexcan.obj
 0001:00001480       ??_C@_1FI@GLCACMKB@?$AAF?$AAl?$AAe?$AAx?$AAC?$AAA?$AAN?$AA?5?$AAD?$AAr?$AAi?$AAv?$AAe?$AAr?$AA?3?$AA?5?$AA?9?$AAF?$AAl?$AAe?$AAx?$AAC?$AAA?$AAN?$AA?3?$AA?3?$AAD?$AAe?$AAi?$AAn?$AAi?$AAt@ 10002480     flexcan.obj
 0001:000014d8       ??_C@_1FI@OADBENNE@?$AAF?$AAl?$AAe?$AAx?$AAC?$AAA?$AAN?$AA?5?$AAD?$AAr?$AAi?$AAv?$AAe?$AAr?$AA?3?$AA?5?$AA?$CL?$AAF?$AAl?$AAe?$AAx?$AAC?$AAA?$AAN?$AA?3?$AA?3?$AAD?$AAe?$AAi?$AAn?$AAi?$AAt@ 100024d8     flexcan.obj
 0001:00001530       ??_C@_1FG@IFIHBBLA@?$AAF?$AAl?$AAe?$AAx?$AAC?$AAA?$AAN?$AA?5?$AAD?$AAr?$AAi?$AAv?$AAe?$AAr?$AA?3?$AA?5?$AA?9?$AAF?$AAl?$AAe?$AAx?$AAC?$AAA?$AAN?$AA?3?$AA?3?$AAI?$AAn?$AAi?$AAt?$AAF?$AAl@ 10002530     flexcan.obj
 0001:00001588       ??_C@_1FG@EGDFONID@?$AAF?$AAl?$AAe?$AAx?$AAC?$AAA?$AAN?$AA?5?$AAD?$AAr?$AAi?$AAv?$AAe?$AAr?$AA?3?$AA?5?$AA?$CL?$AAF?$AAl?$AAe?$AAx?$AAC?$AAA?$AAN?$AA?3?$AA?3?$AAI?$AAn?$AAi?$AAt?$AAF?$AAl@ 10002588     flexcan.obj
 0001:000015e0       ??_C@_1EK@IGFMMPOG@?$AAF?$AAl?$AAe?$AAx?$AAC?$AAA?$AAN?$AA?5?$AAD?$AAr?$AAi?$AAv?$AAe?$AAr?$AA?3?$AA?5?$AA?9?$AAF?$AAl?$AAe?$AAx?$AAC?$AAA?$AAN?$AA?3?$AA?3?$AAI?$AAS?$AAT?$AA?$CI?$AA?$CF?$AAd@ 100025e0     flexcan.obj
 0001:00001630       ??_C@_1FC@HBGKFNBB@?$AAF?$AAl?$AAe?$AAx?$AAC?$AAA?$AAN?$AA?5?$AAD?$AAr?$AAi?$AAv?$AAe?$AAr?$AA?3?$AA?5?$AA?5?$AAF?$AAl?$AAe?$AAx?$AAC?$AAA?$AAN?$AA?3?$AA?3?$AAI?$AAS?$AAT?$AA?$DO?$AA?5?$AAW@ 10002630     flexcan.obj
 0001:00001688       ??_C@_1GI@MDPDBFEA@?$AAF?$AAl?$AAe?$AAx?$AAC?$AAA?$AAN?$AA?5?$AAD?$AAr?$AAi?$AAv?$AAe?$AAr?$AA?3?$AA?5?$AA?5?$AAF?$AAl?$AAe?$AAx?$AAC?$AAA?$AAN?$AA?3?$AA?3?$AAI?$AAS?$AAT?$AA?$DO?$AA?5?$AAE@ 10002688     flexcan.obj
 0001:000016f0       ??_C@_1GI@OONKPGAP@?$AAF?$AAl?$AAe?$AAx?$AAC?$AAA?$AAN?$AA?5?$AAD?$AAr?$AAi?$AAv?$AAe?$AAr?$AA?3?$AA?5?$AA?5?$AAF?$AAl?$AAe?$AAx?$AAC?$AAA?$AAN?$AA?3?$AA?3?$AAI?$AAS?$AAT?$AA?$DO?$AA?5?$AAE@ 100026f0     flexcan.obj
 0001:00001758       ??_C@_1GI@NNAJGNEG@?$AAF?$AAl?$AAe?$AAx?$AAC?$AAA?$AAN?$AA?5?$AAD?$AAr?$AAi?$AAv?$AAe?$AAr?$AA?3?$AA?5?$AA?5?$AAF?$AAl?$AAe?$AAx?$AAC?$AAA?$AAN?$AA?3?$AA?3?$AAI?$AAS?$AAT?$AA?$DO?$AA?5?$AAE@ 10002758     flexcan.obj
 0001:000017c0       ??_C@_1GI@IHMJNHIN@?$AAF?$AAl?$AAe?$AAx?$AAC?$AAA?$AAN?$AA?5?$AAD?$AAr?$AAi?$AAv?$AAe?$AAr?$AA?3?$AA?5?$AA?5?$AAF?$AAl?$AAe?$AAx?$AAC?$AAA?$AAN?$AA?3?$AA?3?$AAI?$AAS?$AAT?$AA?$DO?$AA?5?$AAE@ 100027c0     flexcan.obj
 0001:00001828       ??_C@_1GI@FMMEDBDJ@?$AAF?$AAl?$AAe?$AAx?$AAC?$AAA?$AAN?$AA?5?$AAD?$AAr?$AAi?$AAv?$AAe?$AAr?$AA?3?$AA?5?$AA?5?$AAF?$AAl?$AAe?$AAx?$AAC?$AAA?$AAN?$AA?3?$AA?3?$AAI?$AAS?$AAT?$AA?$DO?$AA?5?$AAE@ 10002828     flexcan.obj
 0001:00001890       ??_C@_1GI@DLAHEOGB@?$AAF?$AAl?$AAe?$AAx?$AAC?$AAA?$AAN?$AA?5?$AAD?$AAr?$AAi?$AAv?$AAe?$AAr?$AA?3?$AA?5?$AA?5?$AAF?$AAl?$AAe?$AAx?$AAC?$AAA?$AAN?$AA?3?$AA?3?$AAI?$AAS?$AAT?$AA?$DO?$AA?5?$AAE@ 10002890     flexcan.obj
 0001:000018f8       ??_C@_1GI@JNKCGOAK@?$AAF?$AAl?$AAe?$AAx?$AAC?$AAA?$AAN?$AA?5?$AAD?$AAr?$AAi?$AAv?$AAe?$AAr?$AA?3?$AA?5?$AA?5?$AAF?$AAl?$AAe?$AAx?$AAC?$AAA?$AAN?$AA?3?$AA?3?$AAI?$AAS?$AAT?$AA?$DO?$AA?5?$AAE@ 100028f8     flexcan.obj
 0001:00001960       ??_C@_1GI@JKBNCPNF@?$AAF?$AAl?$AAe?$AAx?$AAC?$AAA?$AAN?$AA?5?$AAD?$AAr?$AAi?$AAv?$AAe?$AAr?$AA?3?$AA?5?$AA?5?$AAF?$AAl?$AAe?$AAx?$AAC?$AAA?$AAN?$AA?3?$AA?3?$AAI?$AAS?$AAT?$AA?$DO?$AA?5?$AAE@ 10002960     flexcan.obj
 0001:000019c8       ??_C@_1GI@HOMPIPL@?$AAF?$AAl?$AAe?$AAx?$AAC?$AAA?$AAN?$AA?5?$AAD?$AAr?$AAi?$AAv?$AAe?$AAr?$AA?3?$AA?5?$AA?5?$AAF?$AAl?$AAe?$AAx?$AAC?$AAA?$AAN?$AA?3?$AA?3?$AAI?$AAS?$AAT?$AA?$DO?$AA?5?$AAE@ 100029c8     flexcan.obj
 0001:00001a30       ??_C@_1GI@LPCLBONF@?$AAF?$AAl?$AAe?$AAx?$AAC?$AAA?$AAN?$AA?5?$AAD?$AAr?$AAi?$AAv?$AAe?$AAr?$AA?3?$AA?5?$AA?5?$AAF?$AAl?$AAe?$AAx?$AAC?$AAA?$AAN?$AA?3?$AA?3?$AAI?$AAS?$AAT?$AA?$DO?$AA?5?$AAE@ 10002a30     flexcan.obj
 0001:00001a98       ??_C@_1GI@LOJOODMI@?$AAF?$AAl?$AAe?$AAx?$AAC?$AAA?$AAN?$AA?5?$AAD?$AAr?$AAi?$AAv?$AAe?$AAr?$AA?3?$AA?5?$AA?5?$AAF?$AAl?$AAe?$AAx?$AAC?$AAA?$AAN?$AA?3?$AA?3?$AAI?$AAS?$AAT?$AA?$DO?$AA?5?$AAE@ 10002a98     flexcan.obj
 0001:00001b00       ??_C@_1FC@KEBLDBIC@?$AAF?$AAl?$AAe?$AAx?$AAC?$AAA?$AAN?$AA?5?$AAD?$AAr?$AAi?$AAv?$AAe?$AAr?$AA?3?$AA?5?$AA?5?$AAF?$AAl?$AAe?$AAx?$AAC?$AAA?$AAN?$AA?3?$AA?3?$AAI?$AAS?$AAT?$AA?$DO?$AA?5?$AAE@ 10002b00     flexcan.obj
 0001:00001b58       ??_C@_1FE@JHMHMBDL@?$AAF?$AAl?$AAe?$AAx?$AAC?$AAA?$AAN?$AA?5?$AAD?$AAr?$AAi?$AAv?$AAe?$AAr?$AA?3?$AA?5?$AA?5?$AAF?$AAl?$AAe?$AAx?$AAC?$AAA?$AAN?$AA?3?$AA?3?$AAI?$AAS?$AAT?$AA?$DO?$AA?5?$AAB@ 10002b58     flexcan.obj
 0001:00001bb0       ??_C@_1GI@ONNKFJNA@?$AAF?$AAl?$AAe?$AAx?$AAC?$AAA?$AAN?$AA?5?$AAD?$AAr?$AAi?$AAv?$AAe?$AAr?$AA?3?$AA?5?$AA?5?$AAF?$AAl?$AAe?$AAx?$AAC?$AAA?$AAN?$AA?3?$AA?3?$AAI?$AAS?$AAT?$AA?$DO?$AA?5?$AAE@ 10002bb0     flexcan.obj
 0001:00001c18       ??_C@_1FE@BFDFOCLM@?$AAF?$AAl?$AAe?$AAx?$AAC?$AAA?$AAN?$AA?5?$AAD?$AAr?$AAi?$AAv?$AAe?$AAr?$AA?3?$AA?5?$AA?5?$AAF?$AAl?$AAe?$AAx?$AAC?$AAA?$AAN?$AA?3?$AA?3?$AAI?$AAS?$AAT?$AA?$DO?$AA?5?$AAR@ 10002c18     flexcan.obj
 0001:00001c70       ??_C@_1GI@DGNHLPGE@?$AAF?$AAl?$AAe?$AAx?$AAC?$AAA?$AAN?$AA?5?$AAD?$AAr?$AAi?$AAv?$AAe?$AAr?$AA?3?$AA?5?$AA?5?$AAF?$AAl?$AAe?$AAx?$AAC?$AAA?$AAN?$AA?3?$AA?3?$AAI?$AAS?$AAT?$AA?$DO?$AA?5?$AAE@ 10002c70     flexcan.obj
 0001:00001cd8       ??_C@_1FE@GHMELIDM@?$AAF?$AAl?$AAe?$AAx?$AAC?$AAA?$AAN?$AA?5?$AAD?$AAr?$AAi?$AAv?$AAe?$AAr?$AA?3?$AA?5?$AA?5?$AAF?$AAl?$AAe?$AAx?$AAC?$AAA?$AAN?$AA?3?$AA?3?$AAI?$AAS?$AAT?$AA?$DO?$AA?5?$AAT@ 10002cd8     flexcan.obj
 0001:00001d30       ??_C@_1FI@EDAAACDO@?$AAF?$AAl?$AAe?$AAx?$AAC?$AAA?$AAN?$AA?5?$AAD?$AAr?$AAi?$AAv?$AAe?$AAr?$AA?3?$AA?5?$AA?5?$AAF?$AAl?$AAe?$AAx?$AAC?$AAA?$AAN?$AA?3?$AA?3?$AAI?$AAS?$AAT?$AA?$DO?$AA?5?$AAM@ 10002d30     flexcan.obj
 0001:00001d88       ??_C@_1EG@FCGEIPMO@?$AAF?$AAl?$AAe?$AAx?$AAC?$AAA?$AAN?$AA?5?$AAD?$AAr?$AAi?$AAv?$AAe?$AAr?$AA?3?$AA?5?$AA?$CL?$AAF?$AAl?$AAe?$AAx?$AAC?$AAA?$AAN?$AA?3?$AA?3?$AAI?$AAS?$AAT?$AA?$CI?$AA?$CJ?$AA?$CL@ 10002d88     flexcan.obj
 0001:00001dd0       ??_C@_1GO@MDAFHIDD@?$AAF?$AAl?$AAe?$AAx?$AAC?$AAA?$AAN?$AA?5?$AAD?$AAr?$AAi?$AAv?$AAe?$AAr?$AA?3?$AA?5?$AA?9?$AAF?$AAl?$AAe?$AAx?$AAC?$AAA?$AAN?$AA?3?$AA?3?$AAS?$AAe?$AAt?$AAu?$AAp?$AAI@ 10002dd0     flexcan.obj
 0001:00001e40       ??_C@_1LA@NOLEOGOD@?$AAF?$AAl?$AAe?$AAx?$AAC?$AAA?$AAN?$AA?5?$AAD?$AAr?$AAi?$AAv?$AAe?$AAr?$AA?3?$AA?5?$AA?5?$AAF?$AAl?$AAe?$AAx?$AAC?$AAA?$AAN?$AA?3?$AA?3?$AAS?$AAe?$AAt?$AAu?$AAp?$AAI@ 10002e40     flexcan.obj
 0001:00001ef0       ??_C@_1LC@FCLGMELC@?$AAF?$AAl?$AAe?$AAx?$AAC?$AAA?$AAN?$AA?5?$AAD?$AAr?$AAi?$AAv?$AAe?$AAr?$AA?3?$AA?5?$AA?5?$AAF?$AAl?$AAe?$AAx?$AAC?$AAA?$AAN?$AA?3?$AA?3?$AAS?$AAe?$AAt?$AAu?$AAp?$AAI@ 10002ef0     flexcan.obj
 0001:00001fa8       ??_C@_1ME@HHCIEJEB@?$AAF?$AAl?$AAe?$AAx?$AAC?$AAA?$AAN?$AA?5?$AAD?$AAr?$AAi?$AAv?$AAe?$AAr?$AA?3?$AA?5?$AA?5?$AAF?$AAl?$AAe?$AAx?$AAC?$AAA?$AAN?$AA?3?$AA?3?$AAS?$AAe?$AAt?$AAu?$AAp?$AAI@ 10002fa8     flexcan.obj
 0001:00002070       ??_C@_1MM@LFMLEHAK@?$AAF?$AAl?$AAe?$AAx?$AAC?$AAA?$AAN?$AA?5?$AAD?$AAr?$AAi?$AAv?$AAe?$AAr?$AA?3?$AA?5?$AA?5?$AAF?$AAl?$AAe?$AAx?$AAC?$AAA?$AAN?$AA?3?$AA?3?$AAS?$AAe?$AAt?$AAu?$AAp?$AAI@ 10003070     flexcan.obj
 0001:00002140       ??_C@_1MI@CANBPKPJ@?$AAF?$AAl?$AAe?$AAx?$AAC?$AAA?$AAN?$AA?5?$AAD?$AAr?$AAi?$AAv?$AAe?$AAr?$AA?3?$AA?5?$AA?5?$AAF?$AAl?$AAe?$AAx?$AAC?$AAA?$AAN?$AA?3?$AA?3?$AAS?$AAe?$AAt?$AAu?$AAp?$AAI@ 10003140     flexcan.obj
 0001:00002208       ??_C@_1GK@LAKBAHEF@?$AAF?$AAl?$AAe?$AAx?$AAC?$AAA?$AAN?$AA?5?$AAD?$AAr?$AAi?$AAv?$AAe?$AAr?$AA?3?$AA?5?$AA?$CL?$AAF?$AAl?$AAe?$AAx?$AAC?$AAA?$AAN?$AA?3?$AA?3?$AAS?$AAe?$AAt?$AAu?$AAp?$AAI@ 10003208     flexcan.obj
 0001:00002278       ??_C@_1GK@PAPPDOMH@?$AAF?$AAl?$AAe?$AAx?$AAC?$AAA?$AAN?$AA?5?$AAD?$AAr?$AAi?$AAv?$AAe?$AAr?$AA?3?$AA?5?$AA?9?$AAF?$AAl?$AAe?$AAx?$AAC?$AAA?$AAN?$AA?3?$AA?3?$AAC?$AAl?$AAe?$AAa?$AAn?$AAI@ 10003278     flexcan.obj
 0001:000022e8       ??_C@_1GK@IKDHKFJ@?$AAF?$AAl?$AAe?$AAx?$AAC?$AAA?$AAN?$AA?5?$AAD?$AAr?$AAi?$AAv?$AAe?$AAr?$AA?3?$AA?5?$AA?$CL?$AAF?$AAl?$AAe?$AAx?$AAC?$AAA?$AAN?$AA?3?$AA?3?$AAC?$AAl?$AAe?$AAa?$AAn?$AAI@ 100032e8     flexcan.obj
 0001:00002358       ??_C@_1KE@KHMHMNDO@?$AAF?$AAl?$AAe?$AAx?$AAC?$AAA?$AAN?$AA?5?$AAD?$AAr?$AAi?$AAv?$AAe?$AAr?$AA?3?$AA?5?$AA?5?$AAF?$AAl?$AAe?$AAx?$AAC?$AAA?$AAN?$AA?3?$AA?3?$AAS?$AAe?$AAt?$AAB?$AAi?$AAt@ 10003358     flexcan.obj
 0001:00002400       ??_C@_1JO@HOMAPNOK@?$AAF?$AAl?$AAe?$AAx?$AAC?$AAA?$AAN?$AA?5?$AAD?$AAr?$AAi?$AAv?$AAe?$AAr?$AA?3?$AA?5?$AA?5?$AAF?$AAl?$AAe?$AAx?$AAC?$AAA?$AAN?$AA?3?$AA?3?$AAF?$AAi?$AAn?$AAd?$AAF?$AAr@ 10003400     flexcan.obj
 0001:000024a0       ??_C@_1FM@LFLLFFKD@?$AAF?$AAl?$AAe?$AAx?$AAC?$AAA?$AAN?$AA?5?$AAD?$AAr?$AAi?$AAv?$AAe?$AAr?$AA?3?$AA?5?$AA?9?$AAF?$AAl?$AAe?$AAx?$AAC?$AAA?$AAN?$AA?3?$AA?3?$AAC?$AAa?$AAn?$AAc?$AAe?$AAl@ 100034a0     flexcan.obj
 0001:00002500       ??_C@_1HA@PIKCLBMP@?$AAF?$AAl?$AAe?$AAx?$AAC?$AAA?$AAN?$AA?5?$AAD?$AAr?$AAi?$AAv?$AAe?$AAr?$AA?3?$AA?5?$AA?$CL?$AAF?$AAl?$AAe?$AAx?$AAC?$AAA?$AAN?$AA?3?$AA?3?$AAC?$AAa?$AAn?$AAc?$AAe?$AAl@ 10003500     flexcan.obj
 0001:00002570       ??_C@_1GA@OEPFBNCI@?$AAF?$AAl?$AAe?$AAx?$AAC?$AAA?$AAN?$AA?5?$AAD?$AAr?$AAi?$AAv?$AAe?$AAr?$AA?3?$AA?5?$AA?9?$AAF?$AAl?$AAe?$AAx?$AAC?$AAA?$AAN?$AA?3?$AA?3?$AAT?$AAr?$AAa?$AAn?$AAs?$AAm@ 10003570     flexcan.obj
 0001:000025d0       ??_C@_1MC@IDLBPJPJ@?$AAF?$AAl?$AAe?$AAx?$AAC?$AAA?$AAN?$AA?5?$AAD?$AAr?$AAi?$AAv?$AAe?$AAr?$AA?3?$AA?5?$AA?5?$AAF?$AAl?$AAe?$AAx?$AAC?$AAA?$AAN?$AA?3?$AA?3?$AAT?$AAr?$AAa?$AAn?$AAs?$AAm@ 100035d0     flexcan.obj
 0001:00002698       ??_C@_1LI@KDALDJDH@?$AAF?$AAl?$AAe?$AAx?$AAC?$AAA?$AAN?$AA?5?$AAD?$AAr?$AAi?$AAv?$AAe?$AAr?$AA?3?$AA?5?$AA?5?$AAF?$AAl?$AAe?$AAx?$AAC?$AAA?$AAN?$AA?3?$AA?3?$AAT?$AAr?$AAa?$AAn?$AAs?$AAm@ 10003698     flexcan.obj
 0001:00002750       ??_C@_1BBI@KICEJEIJ@?$AAF?$AAl?$AAe?$AAx?$AAC?$AAA?$AAN?$AA?5?$AAD?$AAr?$AAi?$AAv?$AAe?$AAr?$AA?3?$AA?5?$AA?5?$AAF?$AAl?$AAe?$AAx?$AAC?$AAA?$AAN?$AA?3?$AA?3?$AAT?$AAr?$AAa?$AAn?$AAs?$AAm@ 10003750     flexcan.obj
 0001:00002868       ??_C@_1MG@JGKPCKCP@?$AAF?$AAl?$AAe?$AAx?$AAC?$AAA?$AAN?$AA?5?$AAD?$AAr?$AAi?$AAv?$AAe?$AAr?$AA?3?$AA?5?$AA?5?$AAF?$AAl?$AAe?$AAx?$AAC?$AAA?$AAN?$AA?3?$AA?3?$AAT?$AAr?$AAa?$AAn?$AAs?$AAm@ 10003868     flexcan.obj
 0001:00002930       ??_C@_1II@MONJOCKE@?$AAF?$AAl?$AAe?$AAx?$AAC?$AAA?$AAN?$AA?5?$AAD?$AAr?$AAi?$AAv?$AAe?$AAr?$AA?3?$AA?5?$AA?5?$AAF?$AAl?$AAe?$AAx?$AAC?$AAA?$AAN?$AA?3?$AA?3?$AAT?$AAr?$AAa?$AAn?$AAs?$AAm@ 10003930     flexcan.obj
 0001:000029b8       ??_C@_1IC@CHPAGKGE@?$AAF?$AAl?$AAe?$AAx?$AAC?$AAA?$AAN?$AA?5?$AAD?$AAr?$AAi?$AAv?$AAe?$AAr?$AA?3?$AA?5?$AA?$CL?$AAF?$AAl?$AAe?$AAx?$AAC?$AAA?$AAN?$AA?3?$AA?3?$AAT?$AAr?$AAa?$AAn?$AAs?$AAm@ 100039b8     flexcan.obj
 0001:00002a40       ??_C@_1FO@HHMKFKME@?$AAF?$AAl?$AAe?$AAx?$AAC?$AAA?$AAN?$AA?5?$AAD?$AAr?$AAi?$AAv?$AAe?$AAr?$AA?3?$AA?5?$AA?9?$AAF?$AAl?$AAe?$AAx?$AAC?$AAA?$AAN?$AA?3?$AA?3?$AAR?$AAe?$AAc?$AAe?$AAi?$AAv@ 10003a40     flexcan.obj
 0001:00002aa0       ??_C@_1MA@IEOAKLLJ@?$AAF?$AAl?$AAe?$AAx?$AAC?$AAA?$AAN?$AA?5?$AAD?$AAr?$AAi?$AAv?$AAe?$AAr?$AA?3?$AA?5?$AA?5?$AAF?$AAl?$AAe?$AAx?$AAC?$AAA?$AAN?$AA?3?$AA?3?$AAR?$AAe?$AAc?$AAe?$AAi?$AAv@ 10003aa0     flexcan.obj
 0001:00002b60       ??_C@_1LG@FLFJIAOO@?$AAF?$AAl?$AAe?$AAx?$AAC?$AAA?$AAN?$AA?5?$AAD?$AAr?$AAi?$AAv?$AAe?$AAr?$AA?3?$AA?5?$AA?5?$AAF?$AAl?$AAe?$AAx?$AAC?$AAA?$AAN?$AA?3?$AA?3?$AAR?$AAe?$AAc?$AAe?$AAi?$AAv@ 10003b60     flexcan.obj
 0001:00002c18       ??_C@_1BBG@PLNEBOLF@?$AAF?$AAl?$AAe?$AAx?$AAC?$AAA?$AAN?$AA?5?$AAD?$AAr?$AAi?$AAv?$AAe?$AAr?$AA?3?$AA?5?$AA?5?$AAF?$AAl?$AAe?$AAx?$AAC?$AAA?$AAN?$AA?3?$AA?3?$AAR?$AAe?$AAc?$AAe?$AAi?$AAv@ 10003c18     flexcan.obj
 0001:00002d30       ??_C@_1ME@FPEHHBHK@?$AAF?$AAl?$AAe?$AAx?$AAC?$AAA?$AAN?$AA?5?$AAD?$AAr?$AAi?$AAv?$AAe?$AAr?$AA?3?$AA?5?$AA?5?$AAF?$AAl?$AAe?$AAx?$AAC?$AAA?$AAN?$AA?3?$AA?3?$AAR?$AAe?$AAc?$AAe?$AAi?$AAv@ 10003d30     flexcan.obj
 0001:00002df8       ??_C@_1IG@NCLLKCCO@?$AAF?$AAl?$AAe?$AAx?$AAC?$AAA?$AAN?$AA?5?$AAD?$AAr?$AAi?$AAv?$AAe?$AAr?$AA?3?$AA?5?$AA?5?$AAF?$AAl?$AAe?$AAx?$AAC?$AAA?$AAN?$AA?3?$AA?3?$AAR?$AAe?$AAc?$AAe?$AAi?$AAv@ 10003df8     flexcan.obj
 0001:00002e80       ??_C@_1IA@KFJIMAKM@?$AAF?$AAl?$AAe?$AAx?$AAC?$AAA?$AAN?$AA?5?$AAD?$AAr?$AAi?$AAv?$AAe?$AAr?$AA?3?$AA?5?$AA?$CL?$AAF?$AAl?$AAe?$AAx?$AAC?$AAA?$AAN?$AA?3?$AA?3?$AAR?$AAe?$AAc?$AAe?$AAi?$AAv@ 10003e80     flexcan.obj
 0001:00002f00       ??_C@_1FE@GPBPMGOM@?$AAF?$AAl?$AAe?$AAx?$AAC?$AAA?$AAN?$AA?5?$AAD?$AAr?$AAi?$AAv?$AAe?$AAr?$AA?3?$AA?5?$AA?9?$AAF?$AAl?$AAe?$AAx?$AAC?$AAA?$AAN?$AA?3?$AA?3?$AAB?$AAl?$AAi?$AAn?$AAk?$AAL@ 10003f00     flexcan.obj
 0001:00002f58       ??_C@_1IA@ICPBGDIH@?$AAF?$AAl?$AAe?$AAx?$AAC?$AAA?$AAN?$AA?5?$AAD?$AAr?$AAi?$AAv?$AAe?$AAr?$AA?3?$AA?5?$AA?$CL?$AAF?$AAl?$AAe?$AAx?$AAC?$AAA?$AAN?$AA?3?$AA?3?$AAB?$AAl?$AAi?$AAn?$AAk?$AAL@ 10003f58     flexcan.obj
 0001:00002fd8       ??_C@_1II@NJIFDDKO@?$AAF?$AAl?$AAe?$AAx?$AAC?$AAA?$AAN?$AA?5?$AAD?$AAr?$AAi?$AAv?$AAe?$AAr?$AA?3?$AA?5?$AA?5?$AAF?$AAl?$AAe?$AAx?$AAC?$AAA?$AAN?$AA?3?$AA?3?$AAD?$AAu?$AAm?$AAp?$AAR?$AAe@ 10003fd8     flexcan.obj
 0001:00003060       ??_C@_1II@MOKNFHGO@?$AAF?$AAl?$AAe?$AAx?$AAC?$AAA?$AAN?$AA?5?$AAD?$AAr?$AAi?$AAv?$AAe?$AAr?$AA?3?$AA?5?$AA?5?$AAF?$AAl?$AAe?$AAx?$AAC?$AAA?$AAN?$AA?3?$AA?3?$AAD?$AAu?$AAm?$AAp?$AAR?$AAe@ 10004060     flexcan.obj
 0001:000030e8       ??_C@_1II@PHNFPKCO@?$AAF?$AAl?$AAe?$AAx?$AAC?$AAA?$AAN?$AA?5?$AAD?$AAr?$AAi?$AAv?$AAe?$AAr?$AA?3?$AA?5?$AA?5?$AAF?$AAl?$AAe?$AAx?$AAC?$AAA?$AAN?$AA?3?$AA?3?$AAD?$AAu?$AAm?$AAp?$AAR?$AAe@ 100040e8     flexcan.obj
 0001:00003170       ??_C@_1II@OAPNJOOO@?$AAF?$AAl?$AAe?$AAx?$AAC?$AAA?$AAN?$AA?5?$AAD?$AAr?$AAi?$AAv?$AAe?$AAr?$AA?3?$AA?5?$AA?5?$AAF?$AAl?$AAe?$AAx?$AAC?$AAA?$AAN?$AA?3?$AA?3?$AAD?$AAu?$AAm?$AAp?$AAR?$AAe@ 10004170     flexcan.obj
 0001:000031f8       ??_C@_1II@FODDLKFA@?$AAF?$AAl?$AAe?$AAx?$AAC?$AAA?$AAN?$AA?5?$AAD?$AAr?$AAi?$AAv?$AAe?$AAr?$AA?3?$AA?5?$AA?5?$AAF?$AAl?$AAe?$AAx?$AAC?$AAA?$AAN?$AA?3?$AA?3?$AAD?$AAu?$AAm?$AAp?$AAR?$AAe@ 100041f8     flexcan.obj
 0001:00003280       ??_C@_1II@EJBLNOJA@?$AAF?$AAl?$AAe?$AAx?$AAC?$AAA?$AAN?$AA?5?$AAD?$AAr?$AAi?$AAv?$AAe?$AAr?$AA?3?$AA?5?$AA?5?$AAF?$AAl?$AAe?$AAx?$AAC?$AAA?$AAN?$AA?3?$AA?3?$AAD?$AAu?$AAm?$AAp?$AAR?$AAe@ 10004280     flexcan.obj
 0001:00003308       ??_C@_1II@HAGDHDNA@?$AAF?$AAl?$AAe?$AAx?$AAC?$AAA?$AAN?$AA?5?$AAD?$AAr?$AAi?$AAv?$AAe?$AAr?$AA?3?$AA?5?$AA?5?$AAF?$AAl?$AAe?$AAx?$AAC?$AAA?$AAN?$AA?3?$AA?3?$AAD?$AAu?$AAm?$AAp?$AAR?$AAe@ 10004308     flexcan.obj
 0001:00003390       ??_C@_1II@GHELBHBA@?$AAF?$AAl?$AAe?$AAx?$AAC?$AAA?$AAN?$AA?5?$AAD?$AAr?$AAi?$AAv?$AAe?$AAr?$AA?3?$AA?5?$AA?5?$AAF?$AAl?$AAe?$AAx?$AAC?$AAA?$AAN?$AA?3?$AA?3?$AAD?$AAu?$AAm?$AAp?$AAR?$AAe@ 10004390     flexcan.obj
 0001:00003418       ??_C@_1JA@EGEPOEOG@?$AAF?$AAl?$AAe?$AAx?$AAC?$AAA?$AAN?$AA?5?$AAD?$AAr?$AAi?$AAv?$AAe?$AAr?$AA?3?$AA?5?$AA?5?$AAF?$AAl?$AAe?$AAx?$AAC?$AAA?$AAN?$AA?3?$AA?3?$AAD?$AAu?$AAm?$AAp?$AAR?$AAe@ 10004418     flexcan.obj
 0001:000034a8       ??_C@_1JA@MCKOFBNE@?$AAF?$AAl?$AAe?$AAx?$AAC?$AAA?$AAN?$AA?5?$AAD?$AAr?$AAi?$AAv?$AAe?$AAr?$AA?3?$AA?5?$AA?5?$AAF?$AAl?$AAe?$AAx?$AAC?$AAA?$AAN?$AA?3?$AA?3?$AAD?$AAu?$AAm?$AAp?$AAR?$AAe@ 100044a8     flexcan.obj
 0001:00003538       ??_C@_1II@FMANDPAH@?$AAF?$AAl?$AAe?$AAx?$AAC?$AAA?$AAN?$AA?5?$AAD?$AAr?$AAi?$AAv?$AAe?$AAr?$AA?3?$AA?5?$AA?5?$AAF?$AAl?$AAe?$AAx?$AAC?$AAA?$AAN?$AA?3?$AA?3?$AAD?$AAu?$AAm?$AAp?$AAR?$AAe@ 10004538     flexcan.obj
 0001:000035c0       ??_C@_1II@ICNJCJNN@?$AAF?$AAl?$AAe?$AAx?$AAC?$AAA?$AAN?$AA?5?$AAD?$AAr?$AAi?$AAv?$AAe?$AAr?$AA?3?$AA?5?$AA?5?$AAF?$AAl?$AAe?$AAx?$AAC?$AAA?$AAN?$AA?3?$AA?3?$AAD?$AAu?$AAm?$AAp?$AAR?$AAe@ 100045c0     flexcan.obj
 0001:00003648       ??_C@_1II@JEDPFPBF@?$AAF?$AAl?$AAe?$AAx?$AAC?$AAA?$AAN?$AA?5?$AAD?$AAr?$AAi?$AAv?$AAe?$AAr?$AA?3?$AA?5?$AA?5?$AAF?$AAl?$AAe?$AAx?$AAC?$AAA?$AAN?$AA?3?$AA?3?$AAD?$AAu?$AAm?$AAp?$AAR?$AAe@ 10004648     flexcan.obj
 0001:000036d0       ??_C@_1II@FOHKNPGF@?$AAF?$AAl?$AAe?$AAx?$AAC?$AAA?$AAN?$AA?5?$AAD?$AAr?$AAi?$AAv?$AAe?$AAr?$AA?3?$AA?5?$AA?5?$AAF?$AAl?$AAe?$AAx?$AAC?$AAA?$AAN?$AA?3?$AA?3?$AAD?$AAu?$AAm?$AAp?$AAR?$AAe@ 100046d0     flexcan.obj
 0001:00003758       ??_C@_1II@DBLOEBLO@?$AAF?$AAl?$AAe?$AAx?$AAC?$AAA?$AAN?$AA?5?$AAD?$AAr?$AAi?$AAv?$AAe?$AAr?$AA?3?$AA?5?$AA?5?$AAF?$AAl?$AAe?$AAx?$AAC?$AAA?$AAN?$AA?3?$AA?3?$AAD?$AAu?$AAm?$AAp?$AAR?$AAe@ 10004758     flexcan.obj
 0001:000037e0       ??_C@_1II@DDLHJJGM@?$AAF?$AAl?$AAe?$AAx?$AAC?$AAA?$AAN?$AA?5?$AAD?$AAr?$AAi?$AAv?$AAe?$AAr?$AA?3?$AA?5?$AA?5?$AAF?$AAl?$AAe?$AAx?$AAC?$AAA?$AAN?$AA?3?$AA?3?$AAD?$AAu?$AAm?$AAp?$AAR?$AAe@ 100047e0     flexcan.obj
 0001:00003868       ??_C@_1II@MNBAFOEJ@?$AAF?$AAl?$AAe?$AAx?$AAC?$AAA?$AAN?$AA?5?$AAD?$AAr?$AAi?$AAv?$AAe?$AAr?$AA?3?$AA?5?$AA?5?$AAF?$AAl?$AAe?$AAx?$AAC?$AAA?$AAN?$AA?3?$AA?3?$AAD?$AAu?$AAm?$AAp?$AAR?$AAe@ 10004868     flexcan.obj
 0001:000038f0       ??_C@_1JA@OBOPKDK@?$AAF?$AAl?$AAe?$AAx?$AAC?$AAA?$AAN?$AA?5?$AAD?$AAr?$AAi?$AAv?$AAe?$AAr?$AA?3?$AA?5?$AA?5?$AAF?$AAl?$AAe?$AAx?$AAC?$AAA?$AAN?$AA?3?$AA?3?$AAD?$AAu?$AAm?$AAp?$AAR?$AAe@ 100048f0     flexcan.obj
 0001:00003980       ??_C@_1IE@MBNPFGMK@?$AAF?$AAl?$AAe?$AAx?$AAC?$AAA?$AAN?$AA?5?$AAD?$AAr?$AAi?$AAv?$AAe?$AAr?$AA?3?$AA?5?$AA?5?$AAF?$AAl?$AAe?$AAx?$AAC?$AAA?$AAN?$AA?3?$AA?3?$AAD?$AAu?$AAm?$AAp?$AAR?$AAe@ 10004980     flexcan.obj
 0001:00003a08       ??_C@_1IE@OLGDOGEC@?$AAF?$AAl?$AAe?$AAx?$AAC?$AAA?$AAN?$AA?5?$AAD?$AAr?$AAi?$AAv?$AAe?$AAr?$AA?3?$AA?5?$AA?5?$AAF?$AAl?$AAe?$AAx?$AAC?$AAA?$AAN?$AA?3?$AA?3?$AAD?$AAu?$AAm?$AAp?$AAR?$AAe@ 10004a08     flexcan.obj
 0001:00003a90       ??_C@_1IE@NJGNPBGA@?$AAF?$AAl?$AAe?$AAx?$AAC?$AAA?$AAN?$AA?5?$AAD?$AAr?$AAi?$AAv?$AAe?$AAr?$AA?3?$AA?5?$AA?5?$AAF?$AAl?$AAe?$AAx?$AAC?$AAA?$AAN?$AA?3?$AA?3?$AAD?$AAu?$AAm?$AAp?$AAR?$AAe@ 10004a90     flexcan.obj
 0001:00003b18       ??_C@_1IE@PDNBEBOI@?$AAF?$AAl?$AAe?$AAx?$AAC?$AAA?$AAN?$AA?5?$AAD?$AAr?$AAi?$AAv?$AAe?$AAr?$AA?3?$AA?5?$AA?5?$AAF?$AAl?$AAe?$AAx?$AAC?$AAA?$AAN?$AA?3?$AA?3?$AAD?$AAu?$AAm?$AAp?$AAR?$AAe@ 10004b18     flexcan.obj
 0001:00003ba0       ??_C@_1HM@OHEHIHMH@?$AAF?$AAl?$AAe?$AAx?$AAC?$AAA?$AAN?$AA?5?$AAD?$AAr?$AAi?$AAv?$AAe?$AAr?$AA?3?$AA?5?$AA?5?$AAF?$AAl?$AAe?$AAx?$AAC?$AAA?$AAN?$AA?3?$AA?3?$AAD?$AAu?$AAm?$AAp?$AAR?$AAe@ 10004ba0     flexcan.obj
 0001:00003c20       ??_C@_1HM@CLEJJLFF@?$AAF?$AAl?$AAe?$AAx?$AAC?$AAA?$AAN?$AA?5?$AAD?$AAr?$AAi?$AAv?$AAe?$AAr?$AA?3?$AA?5?$AA?5?$AAF?$AAl?$AAe?$AAx?$AAC?$AAA?$AAN?$AA?3?$AA?3?$AAD?$AAu?$AAm?$AAp?$AAR?$AAe@ 10004c20     flexcan.obj
 0001:00003ca0       ??_C@_1HM@CHKOLJPD@?$AAF?$AAl?$AAe?$AAx?$AAC?$AAA?$AAN?$AA?5?$AAD?$AAr?$AAi?$AAv?$AAe?$AAr?$AA?3?$AA?5?$AA?5?$AAF?$AAl?$AAe?$AAx?$AAC?$AAA?$AAN?$AA?3?$AA?3?$AAD?$AAu?$AAm?$AAp?$AAR?$AAe@ 10004ca0     flexcan.obj
 0001:00003d20       ??_C@_1HM@CMAKKEEA@?$AAF?$AAl?$AAe?$AAx?$AAC?$AAA?$AAN?$AA?5?$AAD?$AAr?$AAi?$AAv?$AAe?$AAr?$AA?3?$AA?5?$AA?5?$AAF?$AAl?$AAe?$AAx?$AAC?$AAA?$AAN?$AA?3?$AA?3?$AAD?$AAu?$AAm?$AAp?$AAR?$AAe@ 10004d20     flexcan.obj
 0001:00003da0       ??_C@_1HM@BCDEHAP@?$AAF?$AAl?$AAe?$AAx?$AAC?$AAA?$AAN?$AA?5?$AAD?$AAr?$AAi?$AAv?$AAe?$AAr?$AA?3?$AA?5?$AA?5?$AAF?$AAl?$AAe?$AAx?$AAC?$AAA?$AAN?$AA?3?$AA?3?$AAD?$AAu?$AAm?$AAp?$AAR?$AAe@ 10004da0     flexcan.obj
 0001:00003e20       ??_C@_1HM@DCPANMEG@?$AAF?$AAl?$AAe?$AAx?$AAC?$AAA?$AAN?$AA?5?$AAD?$AAr?$AAi?$AAv?$AAe?$AAr?$AA?3?$AA?5?$AA?5?$AAF?$AAl?$AAe?$AAx?$AAC?$AAA?$AAN?$AA?3?$AA?3?$AAD?$AAu?$AAm?$AAp?$AAR?$AAe@ 10004e20     flexcan.obj
 0001:00003ea0       ??_C@_1HM@GIDAGGIN@?$AAF?$AAl?$AAe?$AAx?$AAC?$AAA?$AAN?$AA?5?$AAD?$AAr?$AAi?$AAv?$AAe?$AAr?$AA?3?$AA?5?$AA?5?$AAF?$AAl?$AAe?$AAx?$AAC?$AAA?$AAN?$AA?3?$AA?3?$AAD?$AAu?$AAm?$AAp?$AAR?$AAe@ 10004ea0     flexcan.obj
 0001:00003f20       ??_C@_1HM@LDDNIADJ@?$AAF?$AAl?$AAe?$AAx?$AAC?$AAA?$AAN?$AA?5?$AAD?$AAr?$AAi?$AAv?$AAe?$AAr?$AA?3?$AA?5?$AA?5?$AAF?$AAl?$AAe?$AAx?$AAC?$AAA?$AAN?$AA?3?$AA?3?$AAD?$AAu?$AAm?$AAp?$AAR?$AAe@ 10004f20     flexcan.obj
 0001:00003fa0       ??_C@_1HM@NEPOPPGB@?$AAF?$AAl?$AAe?$AAx?$AAC?$AAA?$AAN?$AA?5?$AAD?$AAr?$AAi?$AAv?$AAe?$AAr?$AA?3?$AA?5?$AA?5?$AAF?$AAl?$AAe?$AAx?$AAC?$AAA?$AAN?$AA?3?$AA?3?$AAD?$AAu?$AAm?$AAp?$AAR?$AAe@ 10004fa0     flexcan.obj
 0001:00004020       ??_C@_1HM@HCFLNPAK@?$AAF?$AAl?$AAe?$AAx?$AAC?$AAA?$AAN?$AA?5?$AAD?$AAr?$AAi?$AAv?$AAe?$AAr?$AA?3?$AA?5?$AA?5?$AAF?$AAl?$AAe?$AAx?$AAC?$AAA?$AAN?$AA?3?$AA?3?$AAD?$AAu?$AAm?$AAp?$AAR?$AAe@ 10005020     flexcan.obj
 0001:000040a0       ??_C@_1HM@HFOEJONF@?$AAF?$AAl?$AAe?$AAx?$AAC?$AAA?$AAN?$AA?5?$AAD?$AAr?$AAi?$AAv?$AAe?$AAr?$AA?3?$AA?5?$AA?5?$AAF?$AAl?$AAe?$AAx?$AAC?$AAA?$AAN?$AA?3?$AA?3?$AAD?$AAu?$AAm?$AAp?$AAR?$AAe@ 100050a0     flexcan.obj
 0001:00004120       ??_C@_1HM@OIBFEJPL@?$AAF?$AAl?$AAe?$AAx?$AAC?$AAA?$AAN?$AA?5?$AAD?$AAr?$AAi?$AAv?$AAe?$AAr?$AA?3?$AA?5?$AA?5?$AAF?$AAl?$AAe?$AAx?$AAC?$AAA?$AAN?$AA?3?$AA?3?$AAD?$AAu?$AAm?$AAp?$AAR?$AAe@ 10005120     flexcan.obj
 0001:000041a0       ??_C@_1HM@FANCKPNF@?$AAF?$AAl?$AAe?$AAx?$AAC?$AAA?$AAN?$AA?5?$AAD?$AAr?$AAi?$AAv?$AAe?$AAr?$AA?3?$AA?5?$AA?5?$AAF?$AAl?$AAe?$AAx?$AAC?$AAA?$AAN?$AA?3?$AA?3?$AAD?$AAu?$AAm?$AAp?$AAR?$AAe@ 100051a0     flexcan.obj
 0001:00004220       ??_C@_1HM@FBGHFCMI@?$AAF?$AAl?$AAe?$AAx?$AAC?$AAA?$AAN?$AA?5?$AAD?$AAr?$AAi?$AAv?$AAe?$AAr?$AA?3?$AA?5?$AA?5?$AAF?$AAl?$AAe?$AAx?$AAC?$AAA?$AAN?$AA?3?$AA?3?$AAD?$AAu?$AAm?$AAp?$AAR?$AAe@ 10005220     flexcan.obj
 0001:000042a0       ??_C@_1HM@HAJFKCCH@?$AAF?$AAl?$AAe?$AAx?$AAC?$AAA?$AAN?$AA?5?$AAD?$AAr?$AAi?$AAv?$AAe?$AAr?$AA?3?$AA?5?$AA?5?$AAF?$AAl?$AAe?$AAx?$AAC?$AAA?$AAN?$AA?3?$AA?3?$AAD?$AAu?$AAm?$AAp?$AAR?$AAe@ 100052a0     flexcan.obj
 0001:00004320       ??_C@_1HM@KLJIEEJD@?$AAF?$AAl?$AAe?$AAx?$AAC?$AAA?$AAN?$AA?5?$AAD?$AAr?$AAi?$AAv?$AAe?$AAr?$AA?3?$AA?5?$AA?5?$AAF?$AAl?$AAe?$AAx?$AAC?$AAA?$AAN?$AA?3?$AA?3?$AAD?$AAu?$AAm?$AAp?$AAR?$AAe@ 10005320     flexcan.obj
 0001:000043a0       ??_C@_1HM@NJCOAOGE@?$AAF?$AAl?$AAe?$AAx?$AAC?$AAA?$AAN?$AA?5?$AAD?$AAr?$AAi?$AAv?$AAe?$AAr?$AA?3?$AA?5?$AA?5?$AAF?$AAl?$AAe?$AAx?$AAC?$AAA?$AAN?$AA?3?$AA?3?$AAD?$AAu?$AAm?$AAp?$AAR?$AAe@ 100053a0     flexcan.obj
 0001:00004420       ??_C@_1HM@CCDOINA@?$AAF?$AAl?$AAe?$AAx?$AAC?$AAA?$AAN?$AA?5?$AAD?$AAr?$AAi?$AAv?$AAe?$AAr?$AA?3?$AA?5?$AA?5?$AAF?$AAl?$AAe?$AAx?$AAC?$AAA?$AAN?$AA?3?$AA?3?$AAD?$AAu?$AAm?$AAp?$AAR?$AAe@ 10005420     flexcan.obj
 0001:000044a0       ??_C@_1IE@LLJKAICO@?$AAF?$AAl?$AAe?$AAx?$AAC?$AAA?$AAN?$AA?5?$AAD?$AAr?$AAi?$AAv?$AAe?$AAr?$AA?3?$AA?5?$AA?5?$AAF?$AAl?$AAe?$AAx?$AAC?$AAA?$AAN?$AA?3?$AA?3?$AAD?$AAu?$AAm?$AAp?$AAR?$AAe@ 100054a0     flexcan.obj
 0001:00004528       ??_C@_1IE@JBLCDAEM@?$AAF?$AAl?$AAe?$AAx?$AAC?$AAA?$AAN?$AA?5?$AAD?$AAr?$AAi?$AAv?$AAe?$AAr?$AA?3?$AA?5?$AA?5?$AAF?$AAl?$AAe?$AAx?$AAC?$AAA?$AAN?$AA?3?$AA?3?$AAD?$AAu?$AAm?$AAp?$AAR?$AAe@ 10005528     flexcan.obj
 0001:000045b0       ??_C@_1IE@HIKNKON@?$AAF?$AAl?$AAe?$AAx?$AAC?$AAA?$AAN?$AA?5?$AAD?$AAr?$AAi?$AAv?$AAe?$AAr?$AA?3?$AA?5?$AA?5?$AAF?$AAl?$AAe?$AAx?$AAC?$AAA?$AAN?$AA?3?$AA?3?$AAD?$AAu?$AAm?$AAp?$AAR?$AAe@ 100055b0     flexcan.obj
 0001:00004638       ??_C@_1IE@JHNMADAL@?$AAF?$AAl?$AAe?$AAx?$AAC?$AAA?$AAN?$AA?5?$AAD?$AAr?$AAi?$AAv?$AAe?$AAr?$AA?3?$AA?5?$AA?5?$AAF?$AAl?$AAe?$AAx?$AAC?$AAA?$AAN?$AA?3?$AA?3?$AAD?$AAu?$AAm?$AAp?$AAR?$AAe@ 10005638     flexcan.obj
 0001:000046c0       ??_C@_1HM@KGPOFMBA@?$AAF?$AAl?$AAe?$AAx?$AAC?$AAA?$AAN?$AA?5?$AAD?$AAr?$AAi?$AAv?$AAe?$AAr?$AA?3?$AA?5?$AA?5?$AAF?$AAl?$AAe?$AAx?$AAC?$AAA?$AAN?$AA?3?$AA?3?$AAD?$AAu?$AAm?$AAp?$AAR?$AAe@ 100056c0     flexcan.obj
 0001:00004740       ??_C@_1HM@HGBBOFOM@?$AAF?$AAl?$AAe?$AAx?$AAC?$AAA?$AAN?$AA?5?$AAD?$AAr?$AAi?$AAv?$AAe?$AAr?$AA?3?$AA?5?$AA?5?$AAF?$AAl?$AAe?$AAx?$AAC?$AAA?$AAN?$AA?3?$AA?3?$AAD?$AAu?$AAm?$AAp?$AAR?$AAe@ 10005740     flexcan.obj
 0001:000047c0       ??_C@_1HM@OBKFKHNO@?$AAF?$AAl?$AAe?$AAx?$AAC?$AAA?$AAN?$AA?5?$AAD?$AAr?$AAi?$AAv?$AAe?$AAr?$AA?3?$AA?5?$AA?5?$AAF?$AAl?$AAe?$AAx?$AAC?$AAA?$AAN?$AA?3?$AA?3?$AAD?$AAu?$AAm?$AAp?$AAR?$AAe@ 100057c0     flexcan.obj
 0001:00004840       ??_C@_1HM@NDFBDEJ@?$AAF?$AAl?$AAe?$AAx?$AAC?$AAA?$AAN?$AA?5?$AAD?$AAr?$AAi?$AAv?$AAe?$AAr?$AA?3?$AA?5?$AA?5?$AAF?$AAl?$AAe?$AAx?$AAC?$AAA?$AAN?$AA?3?$AA?3?$AAD?$AAu?$AAm?$AAp?$AAR?$AAe@ 10005840     flexcan.obj
 0001:000048c0       ??_C@_1HM@CPCLFEKF@?$AAF?$AAl?$AAe?$AAx?$AAC?$AAA?$AAN?$AA?5?$AAD?$AAr?$AAi?$AAv?$AAe?$AAr?$AA?3?$AA?5?$AA?5?$AAF?$AAl?$AAe?$AAx?$AAC?$AAA?$AAN?$AA?3?$AA?3?$AAD?$AAu?$AAm?$AAp?$AAR?$AAe@ 100058c0     flexcan.obj
 0001:00004940       ??_C@_1HM@FJJKFLIF@?$AAF?$AAl?$AAe?$AAx?$AAC?$AAA?$AAN?$AA?5?$AAD?$AAr?$AAi?$AAv?$AAe?$AAr?$AA?3?$AA?5?$AA?5?$AAF?$AAl?$AAe?$AAx?$AAC?$AAA?$AAN?$AA?3?$AA?3?$AAD?$AAu?$AAm?$AAp?$AAR?$AAe@ 10005940     flexcan.obj
 0001:000049c0       ??_C@_1HM@DEJANKKK@?$AAF?$AAl?$AAe?$AAx?$AAC?$AAA?$AAN?$AA?5?$AAD?$AAr?$AAi?$AAv?$AAe?$AAr?$AA?3?$AA?5?$AA?5?$AAF?$AAl?$AAe?$AAx?$AAC?$AAA?$AAN?$AA?3?$AA?3?$AAD?$AAu?$AAm?$AAp?$AAR?$AAe@ 100059c0     flexcan.obj
 0001:00004a40       ??_C@_1HM@HNNPMNJF@?$AAF?$AAl?$AAe?$AAx?$AAC?$AAA?$AAN?$AA?5?$AAD?$AAr?$AAi?$AAv?$AAe?$AAr?$AA?3?$AA?5?$AA?5?$AAF?$AAl?$AAe?$AAx?$AAC?$AAA?$AAN?$AA?3?$AA?3?$AAD?$AAu?$AAm?$AAp?$AAR?$AAe@ 10005a40     flexcan.obj
 0001:00004ac0       ??_C@_1HM@ICAPHFGM@?$AAF?$AAl?$AAe?$AAx?$AAC?$AAA?$AAN?$AA?5?$AAD?$AAr?$AAi?$AAv?$AAe?$AAr?$AA?3?$AA?5?$AA?5?$AAF?$AAl?$AAe?$AAx?$AAC?$AAA?$AAN?$AA?3?$AA?3?$AAD?$AAu?$AAm?$AAp?$AAR?$AAe@ 10005ac0     flexcan.obj
 0001:00004b40       ??_C@_1HM@LKJOGPMD@?$AAF?$AAl?$AAe?$AAx?$AAC?$AAA?$AAN?$AA?5?$AAD?$AAr?$AAi?$AAv?$AAe?$AAr?$AA?3?$AA?5?$AA?5?$AAF?$AAl?$AAe?$AAx?$AAC?$AAA?$AAN?$AA?3?$AA?3?$AAD?$AAu?$AAm?$AAp?$AAR?$AAe@ 10005b40     flexcan.obj
 0001:00004bc0       ??_C@_1HM@LCOEHHEL@?$AAF?$AAl?$AAe?$AAx?$AAC?$AAA?$AAN?$AA?5?$AAD?$AAr?$AAi?$AAv?$AAe?$AAr?$AA?3?$AA?5?$AA?5?$AAF?$AAl?$AAe?$AAx?$AAC?$AAA?$AAN?$AA?3?$AA?3?$AAD?$AAu?$AAm?$AAp?$AAR?$AAe@ 10005bc0     flexcan.obj
 0001:00004c40       ??_C@_1HM@CJPCJOFI@?$AAF?$AAl?$AAe?$AAx?$AAC?$AAA?$AAN?$AA?5?$AAD?$AAr?$AAi?$AAv?$AAe?$AAr?$AA?3?$AA?5?$AA?5?$AAF?$AAl?$AAe?$AAx?$AAC?$AAA?$AAN?$AA?3?$AA?3?$AAD?$AAu?$AAm?$AAp?$AAR?$AAe@ 10005c40     flexcan.obj
 0001:00004cc0       ??_C@_1HM@HIPMPMDG@?$AAF?$AAl?$AAe?$AAx?$AAC?$AAA?$AAN?$AA?5?$AAD?$AAr?$AAi?$AAv?$AAe?$AAr?$AA?3?$AA?5?$AA?5?$AAF?$AAl?$AAe?$AAx?$AAC?$AAA?$AAN?$AA?3?$AA?3?$AAD?$AAu?$AAm?$AAp?$AAR?$AAe@ 10005cc0     flexcan.obj
 0001:00004d40       ??_C@_1HM@CAOCFFBO@?$AAF?$AAl?$AAe?$AAx?$AAC?$AAA?$AAN?$AA?5?$AAD?$AAr?$AAi?$AAv?$AAe?$AAr?$AA?3?$AA?5?$AA?5?$AAF?$AAl?$AAe?$AAx?$AAC?$AAA?$AAN?$AA?3?$AA?3?$AAD?$AAu?$AAm?$AAp?$AAR?$AAe@ 10005d40     flexcan.obj
 0001:00004dc0       ??_C@_1HM@BJGLAEEE@?$AAF?$AAl?$AAe?$AAx?$AAC?$AAA?$AAN?$AA?5?$AAD?$AAr?$AAi?$AAv?$AAe?$AAr?$AA?3?$AA?5?$AA?5?$AAF?$AAl?$AAe?$AAx?$AAC?$AAA?$AAN?$AA?3?$AA?3?$AAD?$AAu?$AAm?$AAp?$AAR?$AAe@ 10005dc0     flexcan.obj
 0001:00004e40       ??_C@_1HM@HEFNMOBD@?$AAF?$AAl?$AAe?$AAx?$AAC?$AAA?$AAN?$AA?5?$AAD?$AAr?$AAi?$AAv?$AAe?$AAr?$AA?3?$AA?5?$AA?5?$AAF?$AAl?$AAe?$AAx?$AAC?$AAA?$AAN?$AA?3?$AA?3?$AAD?$AAu?$AAm?$AAp?$AAR?$AAe@ 10005e40     flexcan.obj
 0001:00004ec0       ??_C@_1HM@PFAHEGA@?$AAF?$AAl?$AAe?$AAx?$AAC?$AAA?$AAN?$AA?5?$AAD?$AAr?$AAi?$AAv?$AAe?$AAr?$AA?3?$AA?5?$AA?5?$AAF?$AAl?$AAe?$AAx?$AAC?$AAA?$AAN?$AA?3?$AA?3?$AAD?$AAu?$AAm?$AAp?$AAR?$AAe@ 10005ec0     flexcan.obj
 0001:00004f40       ??_C@_1HM@DHLGHCMO@?$AAF?$AAl?$AAe?$AAx?$AAC?$AAA?$AAN?$AA?5?$AAD?$AAr?$AAi?$AAv?$AAe?$AAr?$AA?3?$AA?5?$AA?5?$AAF?$AAl?$AAe?$AAx?$AAC?$AAA?$AAN?$AA?3?$AA?3?$AAD?$AAu?$AAm?$AAp?$AAR?$AAe@ 10005f40     flexcan.obj
 0001:00004fc0       ??_C@_1HM@OFFGEKMN@?$AAF?$AAl?$AAe?$AAx?$AAC?$AAA?$AAN?$AA?5?$AAD?$AAr?$AAi?$AAv?$AAe?$AAr?$AA?3?$AA?5?$AA?5?$AAF?$AAl?$AAe?$AAx?$AAC?$AAA?$AAN?$AA?3?$AA?3?$AAD?$AAu?$AAm?$AAp?$AAR?$AAe@ 10005fc0     flexcan.obj
 0001:00005040       ??_C@_1HM@GCEBPCAA@?$AAF?$AAl?$AAe?$AAx?$AAC?$AAA?$AAN?$AA?5?$AAD?$AAr?$AAi?$AAv?$AAe?$AAr?$AA?3?$AA?5?$AA?5?$AAF?$AAl?$AAe?$AAx?$AAC?$AAA?$AAN?$AA?3?$AA?3?$AAD?$AAu?$AAm?$AAp?$AAR?$AAe@ 10006040     flexcan.obj
 0001:000050c0       ??_C@_1HM@DEAKNPIB@?$AAF?$AAl?$AAe?$AAx?$AAC?$AAA?$AAN?$AA?5?$AAD?$AAr?$AAi?$AAv?$AAe?$AAr?$AA?3?$AA?5?$AA?5?$AAF?$AAl?$AAe?$AAx?$AAC?$AAA?$AAN?$AA?3?$AA?3?$AAD?$AAu?$AAm?$AAp?$AAR?$AAe@ 100060c0     flexcan.obj
 0001:00005140       ??_C@_1HM@KEFIJPNI@?$AAF?$AAl?$AAe?$AAx?$AAC?$AAA?$AAN?$AA?5?$AAD?$AAr?$AAi?$AAv?$AAe?$AAr?$AA?3?$AA?5?$AA?5?$AAF?$AAl?$AAe?$AAx?$AAC?$AAA?$AAN?$AA?3?$AA?3?$AAD?$AAu?$AAm?$AAp?$AAR?$AAe@ 10006140     flexcan.obj
 0001:000051c0       ??_C@_1HM@FFMBDLMJ@?$AAF?$AAl?$AAe?$AAx?$AAC?$AAA?$AAN?$AA?5?$AAD?$AAr?$AAi?$AAv?$AAe?$AAr?$AA?3?$AA?5?$AA?5?$AAF?$AAl?$AAe?$AAx?$AAC?$AAA?$AAN?$AA?3?$AA?3?$AAD?$AAu?$AAm?$AAp?$AAR?$AAe@ 100061c0     flexcan.obj
 0001:00005240       ??_C@_1HM@PIEECEPI@?$AAF?$AAl?$AAe?$AAx?$AAC?$AAA?$AAN?$AA?5?$AAD?$AAr?$AAi?$AAv?$AAe?$AAr?$AA?3?$AA?5?$AA?5?$AAF?$AAl?$AAe?$AAx?$AAC?$AAA?$AAN?$AA?3?$AA?3?$AAD?$AAu?$AAm?$AAp?$AAR?$AAe@ 10006240     flexcan.obj
 0001:000052c0       ??_C@_1HM@NCMDEMIO@?$AAF?$AAl?$AAe?$AAx?$AAC?$AAA?$AAN?$AA?5?$AAD?$AAr?$AAi?$AAv?$AAe?$AAr?$AA?3?$AA?5?$AA?5?$AAF?$AAl?$AAe?$AAx?$AAC?$AAA?$AAN?$AA?3?$AA?3?$AAD?$AAu?$AAm?$AAp?$AAR?$AAe@ 100062c0     flexcan.obj
 0001:00005340       ??_C@_1HM@FFFAOLNG@?$AAF?$AAl?$AAe?$AAx?$AAC?$AAA?$AAN?$AA?5?$AAD?$AAr?$AAi?$AAv?$AAe?$AAr?$AA?3?$AA?5?$AA?5?$AAF?$AAl?$AAe?$AAx?$AAC?$AAA?$AAN?$AA?3?$AA?3?$AAD?$AAu?$AAm?$AAp?$AAR?$AAe@ 10006340     flexcan.obj
 0001:000053c0       ??_C@_1HM@EIDOFMBG@?$AAF?$AAl?$AAe?$AAx?$AAC?$AAA?$AAN?$AA?5?$AAD?$AAr?$AAi?$AAv?$AAe?$AAr?$AA?3?$AA?5?$AA?5?$AAF?$AAl?$AAe?$AAx?$AAC?$AAA?$AAN?$AA?3?$AA?3?$AAD?$AAu?$AAm?$AAp?$AAR?$AAe@ 100063c0     flexcan.obj
 0001:00005440       ??_C@_1HM@BAEGMMKG@?$AAF?$AAl?$AAe?$AAx?$AAC?$AAA?$AAN?$AA?5?$AAD?$AAr?$AAi?$AAv?$AAe?$AAr?$AA?3?$AA?5?$AA?5?$AAF?$AAl?$AAe?$AAx?$AAC?$AAA?$AAN?$AA?3?$AA?3?$AAD?$AAu?$AAm?$AAp?$AAR?$AAe@ 10006440     flexcan.obj
 0001:000054c0       ??_C@_1HM@JJKPPJDM@?$AAF?$AAl?$AAe?$AAx?$AAC?$AAA?$AAN?$AA?5?$AAD?$AAr?$AAi?$AAv?$AAe?$AAr?$AA?3?$AA?5?$AA?5?$AAF?$AAl?$AAe?$AAx?$AAC?$AAA?$AAN?$AA?3?$AA?3?$AAD?$AAu?$AAm?$AAp?$AAR?$AAe@ 100064c0     flexcan.obj
 0001:00005540       ??_C@_1HM@GNJHJMOP@?$AAF?$AAl?$AAe?$AAx?$AAC?$AAA?$AAN?$AA?5?$AAD?$AAr?$AAi?$AAv?$AAe?$AAr?$AA?3?$AA?5?$AA?5?$AAF?$AAl?$AAe?$AAx?$AAC?$AAA?$AAN?$AA?3?$AA?3?$AAD?$AAu?$AAm?$AAp?$AAR?$AAe@ 10006540     flexcan.obj
 0001:000055c0       ??_C@_1HM@IHMMKK@?$AAF?$AAl?$AAe?$AAx?$AAC?$AAA?$AAN?$AA?5?$AAD?$AAr?$AAi?$AAv?$AAe?$AAr?$AA?3?$AA?5?$AA?5?$AAF?$AAl?$AAe?$AAx?$AAC?$AAA?$AAN?$AA?3?$AA?3?$AAD?$AAu?$AAm?$AAp?$AAR?$AAe@ 100065c0     flexcan.obj
 0001:00005640       ??_C@_1HM@EHFPGFPH@?$AAF?$AAl?$AAe?$AAx?$AAC?$AAA?$AAN?$AA?5?$AAD?$AAr?$AAi?$AAv?$AAe?$AAr?$AA?3?$AA?5?$AA?5?$AAF?$AAl?$AAe?$AAx?$AAC?$AAA?$AAN?$AA?3?$AA?3?$AAD?$AAu?$AAm?$AAp?$AAR?$AAe@ 10006640     flexcan.obj
 0001:000056c0       ??_C@_1HM@HBLEIJHE@?$AAF?$AAl?$AAe?$AAx?$AAC?$AAA?$AAN?$AA?5?$AAD?$AAr?$AAi?$AAv?$AAe?$AAr?$AA?3?$AA?5?$AA?5?$AAF?$AAl?$AAe?$AAx?$AAC?$AAA?$AAN?$AA?3?$AA?3?$AAD?$AAu?$AAm?$AAp?$AAR?$AAe@ 100066c0     flexcan.obj
 0001:00005740       ??_C@_1HM@BKNJPNEP@?$AAF?$AAl?$AAe?$AAx?$AAC?$AAA?$AAN?$AA?5?$AAD?$AAr?$AAi?$AAv?$AAe?$AAr?$AA?3?$AA?5?$AA?5?$AAF?$AAl?$AAe?$AAx?$AAC?$AAA?$AAN?$AA?3?$AA?3?$AAD?$AAu?$AAm?$AAp?$AAR?$AAe@ 10006740     flexcan.obj
 0001:000057c0       ??_C@_1HM@DOHKDBBB@?$AAF?$AAl?$AAe?$AAx?$AAC?$AAA?$AAN?$AA?5?$AAD?$AAr?$AAi?$AAv?$AAe?$AAr?$AA?3?$AA?5?$AA?5?$AAF?$AAl?$AAe?$AAx?$AAC?$AAA?$AAN?$AA?3?$AA?3?$AAD?$AAu?$AAm?$AAp?$AAR?$AAe@ 100067c0     flexcan.obj
 0001:00005840       ??_C@_1HM@IOIFBPGB@?$AAF?$AAl?$AAe?$AAx?$AAC?$AAA?$AAN?$AA?5?$AAD?$AAr?$AAi?$AAv?$AAe?$AAr?$AA?3?$AA?5?$AA?5?$AAF?$AAl?$AAe?$AAx?$AAC?$AAA?$AAN?$AA?3?$AA?3?$AAD?$AAu?$AAm?$AAp?$AAR?$AAe@ 10006840     flexcan.obj
 0001:000058bc       ??_C@_1BA@MNOLBALH@?$AAB?$AAi?$AAt?$AAr?$AAa?$AAt?$AAe?$AA?$AA@ 100068bc     settings.obj
 0001:000058cc       ??_C@_1BI@BHLBGEOK@?$AAP?$AAr?$AAi?$AAo?$AAr?$AAi?$AAt?$AAy?$AA2?$AA5?$AA6?$AA?$AA@ 100068cc     settings.obj
 0001:000058e4       ??_C@_1M@KEKDJCFI@?$AA?$CF?$AAs?$AA?$CF?$AAd?$AA?3?$AA?$AA@ 100068e4     settings.obj
 0001:000058f0       ??_C@_1O@GBAEOCCH@?$AAP?$AAr?$AAe?$AAf?$AAi?$AAx?$AA?$AA@ 100068f0     settings.obj
 0001:00005900       ??_C@_1M@EENNDIOJ@?$AAI?$AAn?$AAd?$AAe?$AAx?$AA?$AA@ 10006900     settings.obj
 0001:00005910       ?canSetup@FlexCAN@@0QBUCAN_SETUP@@B 10006910     flexcan_pdd:pdd.obj
 0001:00005a40       ??_C@_1LK@IOPHFNNJ@?$AAF?$AAl?$AAe?$AAx?$AAC?$AAA?$AAN?$AA?5?$AAD?$AAr?$AAi?$AAv?$AAe?$AAr?$AA?3?$AA?5?$AA?5?$AAF?$AAl?$AAe?$AAx?$AAC?$AAA?$AAN?$AA?3?$AA?3?$AAS?$AAe?$AAt?$AAu?$AAp?$AAH@ 10006a40     flexcan_pdd:pdd.obj
 0001:00005b00       ??_C@_1GA@LHFIGCA@?$AAF?$AAl?$AAe?$AAx?$AAC?$AAA?$AAN?$AA?5?$AAD?$AAr?$AAi?$AAv?$AAe?$AAr?$AA?3?$AA?5?$AA?9?$AAF?$AAl?$AAe?$AAx?$AAC?$AAA?$AAN?$AA?3?$AA?3?$AAL?$AAE?$AAD?$AAB?$AAl?$AAi@ 10006b00     flexcan_pdd:pdd.obj
 0001:00005b60       ??_C@_1FE@NMIGIADD@?$AAF?$AAl?$AAe?$AAx?$AAC?$AAA?$AAN?$AA?5?$AAD?$AAr?$AAi?$AAv?$AAe?$AAr?$AA?3?$AA?5?$AA?$CL?$AAF?$AAl?$AAe?$AAx?$AAC?$AAA?$AAN?$AA?3?$AA?3?$AAL?$AAE?$AAD?$AAB?$AAl?$AAi@ 10006b60     flexcan_pdd:pdd.obj
 0001:00005bd8       ?to_T@@YAPBGPBD@Z          10006bd8 f   DebugZones.obj
 0001:00005c78       DllMain                    10006c78 f   driver.obj
 0001:00005d30       ?Init@@YAPAUDRIVER_INFO@@PAX@Z 10006d30 f   driver.obj
 0001:00005f84       ?Deinit@@YAHPAUDRIVER_INFO@@@Z 10006f84 f   driver.obj
 0001:000060e0       ?Open@@YAPAUOPEN_INFO@@PAUDRIVER_INFO@@KK@Z 100070e0 f   driver.obj
 0001:00006314       ?PreClose@@YAHPAUOPEN_INFO@@@Z 10007314 f   driver.obj
 0001:0000645c       ?Close@@YAHPAUOPEN_INFO@@@Z 1000745c f   driver.obj
 0001:000065c8       ?Read@@YAKPAUOPEN_INFO@@PAEK@Z 100075c8 f   driver.obj
 0001:00006664       ?Write@@YAKPAUOPEN_INFO@@PAEK@Z 10007664 f   driver.obj
 0001:00006700       ?Seek@@YAKPAUOPEN_INFO@@JK@Z 10007700 f   driver.obj
 0001:00006874       ?IOControl@@YAHPAUOPEN_INFO@@KPAEK1KPAK@Z 10007874 f   driver.obj
 0001:00007008       ?IsInitialized@FlexCAN@@QAAHXZ 10008008 f i driver.obj
 0001:00007034       ??_GFlexCAN@@QAAPAXI@Z     10008034 f i driver.obj
 0001:00007078       ??1MarshalledBuffer_t@@QAA@XZ 10008078 f i driver.obj
 0001:00007094       ??0MarshalledBuffer_t@@QAA@PAXKKHH@Z 10008094 f i driver.obj
 0001:000070e8       ?Reset@MarshalledBuffer_t@@AAAXXZ 100080e8 f i driver.obj
 0001:00007128       ?Marshal@MarshalledBuffer_t@@QAAJPAXKKHH@Z 10008128 f i driver.obj
 0001:0000722c       ?Unmarshal@MarshalledBuffer_t@@QAAJXZ 1000822c f i driver.obj
 0001:000072fc       ?ptr@MarshalledBuffer_t@@QBAPAXXZ 100082fc f i driver.obj
 0001:0000734c       ??0?$Buffer_t@VDuplicateTraits_t@detail@marshal@ce@@@detail@marshal@ce@@QAA@PAXKK@Z 1000834c f i driver.obj
 0001:000073a0       ?ptr@?$Buffer_t@VDuplicateTraits_t@detail@marshal@ce@@@detail@marshal@ce@@QBAPAXXZ 100083a0 f i driver.obj
 0001:000073d0       ??1?$Buffer_t@VDuplicateTraits_t@detail@marshal@ce@@@detail@marshal@ce@@UAA@XZ 100083d0 f i driver.obj
 0001:000073fc       ??_G?$Buffer_t@VDuplicateTraits_t@detail@marshal@ce@@@detail@marshal@ce@@UAAPAXI@Z 100083fc f i driver.obj
 0001:000073fc       ??_E?$Buffer_t@VDuplicateTraits_t@detail@marshal@ce@@@detail@marshal@ce@@UAAPAXI@Z 100083fc f i driver.obj
 0001:00007440       ?Reset@?$Buffer_t@VDuplicateTraits_t@detail@marshal@ce@@@detail@marshal@ce@@AAAXXZ 10008440 f i driver.obj
 0001:00007484       ?Free@?$Buffer_t@VDuplicateTraits_t@detail@marshal@ce@@@detail@marshal@ce@@QAAJXZ 10008484 f i driver.obj
 0001:00007520       ?free@DuplicateTraits_t@detail@marshal@ce@@QBAJPAX0KK@Z 10008520 f i driver.obj
 0001:00007560       ?Allocate@?$Buffer_t@VDuplicateTraits_t@detail@marshal@ce@@@detail@marshal@ce@@QAAJPAXKK@Z 10008560 f i driver.obj
 0001:00007614       ?alloc@DuplicateTraits_t@detail@marshal@ce@@QBAJPAPAXPAXKK@Z 10008614 f i driver.obj
 0001:00007654       ??0FlexCAN@@QAA@PBG@Z      10008654 f   flexcan.obj
 0001:000076d8       ??1FlexCAN@@QAA@XZ         100086d8 f   flexcan.obj
 0001:000076f4       ?Initialize@FlexCAN@@AAAHPBG@Z 100086f4 f   flexcan.obj
 0001:00007c74       ?Deinitialize@FlexCAN@@AAAXXZ 10008c74 f   flexcan.obj
 0001:00007f54       ?InitFlexCAN@FlexCAN@@AAAXXZ 10008f54 f   flexcan.obj
 0001:00008520       ?IST@FlexCAN@@CAKPAX@Z     10009520 f   flexcan.obj
 0001:00008dcc       ?SetupInterruptHandler@FlexCAN@@AAAHXZ 10009dcc f   flexcan.obj
 0001:000091c0       ?CleanInterruptHandler@FlexCAN@@AAAXXZ 1000a1c0 f   flexcan.obj
 0001:00009370       ?GetBitrate@FlexCAN@@QAAKXZ 1000a370 f   flexcan.obj
 0001:00009414       ?SetBitrate@FlexCAN@@QAAKK@Z 1000a414 f   flexcan.obj
 0001:000095fc       ?GetCLKSourceFreq@FlexCAN@@AAAKXZ 1000a5fc f   flexcan.obj
 0001:00009660       ?GetClockFreq@FlexCAN@@AAAKXZ 1000a660 f   flexcan.obj
 0001:000096cc       ?EnableMBInterrupt@FlexCAN@@AAAXE@Z 1000a6cc f   flexcan.obj
 0001:000096f0       ?DisableMBInterrupt@FlexCAN@@AAAXE@Z 1000a6f0 f   flexcan.obj
 0001:00009714       ?EnableMBInterrupt@FlexCAN@@AAAXEH@Z 1000a714 f   flexcan.obj
 0001:00009838       ?Swap@FlexCAN@@AAAGG@Z     1000a838 f   flexcan.obj
 0001:00009880       ?Swap@FlexCAN@@AAAKK@Z     1000a880 f   flexcan.obj
 0001:000098e0       ?AbortTransmission@FlexCAN@@AAAKE@Z 1000a8e0 f   flexcan.obj
 0001:00009b6c       ?FindFreeMB@FlexCAN@@AAAEXZ 1000ab6c f   flexcan.obj
 0001:00009c7c       ?CancelPacket@FlexCAN@@QAAKE@Z 1000ac7c f   flexcan.obj
 0001:00009d7c       ?TransmitPacket@FlexCAN@@QAAKPAUCAN_PACKET@@@Z 1000ad7c f   flexcan.obj
 0001:0000a918       ?ReadMessageBuffer@FlexCAN@@AAAHPAUCAN_PACKET@@@Z 1000b918 f   flexcan.obj
 0001:0000ad04       ?ReceivePacket@FlexCAN@@QAAKPAUCAN_PACKET@@@Z 1000bd04 f   flexcan.obj
 0001:0000b3b4       ?SetRxMask@FlexCAN@@AAAXEK@Z 1000c3b4 f   flexcan.obj
 0001:0000b40c       ?EnableDoze@FlexCAN@@QAAXH@Z 1000c40c f   flexcan.obj
 0001:0000b4c0       ?DozeEnabled@FlexCAN@@QAAHXZ 1000c4c0 f   flexcan.obj
 0001:0000b534       ?BlinkLED@FlexCAN@@AAAHW4CAN_LEDS@@K@Z 1000c534 f   flexcan.obj
 0001:0000b7e0       ?DumpRegisters@FlexCAN@@AAAXXZ 1000c7e0 f   flexcan.obj
 0001:0000cd04       ?settingsOK@Settings@@QAAHXZ 1000dd04 f i flexcan.obj
 0001:0000cd30       ?index@Settings@@QAAKXZ    1000dd30 f i flexcan.obj
 0001:0000cd60       ?name@Settings@@QAAPBGXZ   1000dd60 f i flexcan.obj
 0001:0000cd8c       PulseEvent                 1000dd8c f i flexcan.obj
 0001:0000cdc4       ??_GSettings@@QAAPAXI@Z    1000ddc4 f i flexcan.obj
 0001:0000ce08       ?bitrate@Settings@@QAAKXZ  1000de08 f i flexcan.obj
 0001:0000ce38       ?FreezeMode@FlexCAN@@AAAXH@Z 1000de38 f i flexcan.obj
 0001:0000cecc       GetCurrentThread           1000decc f i flexcan.obj
 0001:0000cee4       ?priority256@Settings@@QAAKXZ 1000dee4 f i flexcan.obj
 0001:0000cf14       SetEvent                   1000df14 f i flexcan.obj
 0001:0000cf54       ??0Settings@@QAA@PBG@Z     1000df54 f   settings.obj
 0001:0000d138       ??1Settings@@QAA@XZ        1000e138 f   settings.obj
 0001:0000d14c       ?SetupHardware@FlexCAN@@AAAHK@Z 1000e14c f   flexcan_pdd:pdd.obj
 0001:0000d774       ?LEDBlinker@FlexCAN@@CAKPAX@Z 1000e774 f   flexcan_pdd:pdd.obj
 0001:0000d8dc       RegisterDbgZones           1000e8dc f   coredll:COREDLL.dll
 0001:0000d8ec       DisableThreadLibraryCalls  1000e8ec f   coredll:COREDLL.dll
 0001:0000d8fc       NKDbgPrintfW               1000e8fc f   coredll:COREDLL.dll
 0001:0000d90c       GetLastError               1000e90c f   coredll:COREDLL.dll
 0001:0000d91c       SetLastError               1000e91c f   coredll:COREDLL.dll
 0001:0000d92c       CeAllocAsynchronousBuffer  1000e92c f   coredll:COREDLL.dll
 0001:0000d93c       CeOpenCallerBuffer         1000e93c f   coredll:COREDLL.dll
 0001:0000d94c       CeCloseCallerBuffer        1000e94c f   coredll:COREDLL.dll
 0001:0000d95c       CeFreeAsynchronousBuffer   1000e95c f   coredll:COREDLL.dll
 0001:0000d96c       CeFreeDuplicateBuffer      1000e96c f   coredll:COREDLL.dll
 0001:0000d97c       CeAllocDuplicateBuffer     1000e97c f   coredll:COREDLL.dll
 0001:0000d98c       CreateEventW               1000e98c f   coredll:COREDLL.dll
 0001:0000d99c       InitializeCriticalSection  1000e99c f   coredll:COREDLL.dll
 0001:0000d9ac       CloseHandle                1000e9ac f   coredll:COREDLL.dll
 0001:0000d9bc       TerminateThread            1000e9bc f   coredll:COREDLL.dll
 0001:0000d9cc       WaitForSingleObject        1000e9cc f   coredll:COREDLL.dll
 0001:0000d9dc       DeleteCriticalSection      1000e9dc f   coredll:COREDLL.dll
 0001:0000d9ec       EventModify                1000e9ec f   coredll:COREDLL.dll
 0001:0000d9fc       InterruptDone              1000e9fc f   coredll:COREDLL.dll
 0001:0000da0c       DevicePowerNotify          1000ea0c f   coredll:COREDLL.dll
 0001:0000da1c       CeSetThreadPriority        1000ea1c f   coredll:COREDLL.dll
 0001:0000da2c       CreateThread               1000ea2c f   coredll:COREDLL.dll
 0001:0000da3c       InterruptInitialize        1000ea3c f   coredll:COREDLL.dll
 0001:0000da4c       KernelIoControl            1000ea4c f   coredll:COREDLL.dll
 0001:0000da5c       InterruptDisable           1000ea5c f   coredll:COREDLL.dll
 0001:0000da6c       LeaveCriticalSection       1000ea6c f   coredll:COREDLL.dll
 0001:0000da7c       EnterCriticalSection       1000ea7c f   coredll:COREDLL.dll
 0001:0000da8c       RegCloseKey                1000ea8c f   coredll:COREDLL.dll
 0001:0000da9c       wsprintfW                  1000ea9c f   coredll:COREDLL.dll
 0001:0000daac       RegQueryValueExW           1000eaac f   coredll:COREDLL.dll
 0001:0000dabc       OpenDeviceKey              1000eabc f   coredll:COREDLL.dll
 0001:0000dacc       MmUnmapIoSpace             1000eacc f   ceddk:CEDDK.dll
 0001:0000dadc       MmMapIoSpace               1000eadc f   ceddk:CEDDK.dll
 0001:0000daec       DDKGpioWriteDataPin        1000eaec f   cspddk:CSPDDK.dll
 0001:0000dafc       DDKGpioSetConfig           1000eafc f   cspddk:CSPDDK.dll
 0001:0000db0c       DDKClockSetGatingMode      1000eb0c f   cspddk:CSPDDK.dll
 0001:0000db1c       DDKIomuxSelectInput        1000eb1c f   cspddk:CSPDDK.dll
 0001:0000db2c       DDKIomuxSetPadConfig       1000eb2c f   cspddk:CSPDDK.dll
 0001:0000db3c       DDKIomuxSetPinMux          1000eb3c f   cspddk:CSPDDK.dll
 0001:0000db4c       _DllMainCRTStartup         1000eb4c f   corelib0:pegdmain.obj
 0001:0000dcf4       __security_init_cookie     1000ecf4 f   corelib0:seccinit.obj
 0001:0000ddbc       __GSHandlerCheck           1000edbc f   corelib0:gshandler.obj
 0001:0000de04       __GSHandlerCheckCommon     1000ee04 f   corelib0:gshandler.obj
 0001:0000deac       __security_check_cookie    1000eeac f   corelib0:armsecgs.obj
 0001:0000dec0       __gsfailure                1000eec0 f   corelib0:armsecgs.obj
 0001:0000df04       exit                       1000ef04 f   corelib0:cexit.obj
 0001:0000e084       _exit                      1000f084 f   corelib0:cexit.obj
 0001:0000e0a8       _cexit                     1000f0a8 f   corelib0:cexit.obj
 0001:0000e0c4       _c_exit                    1000f0c4 f   corelib0:cexit.obj
 0001:0000e0e0       GetCurrentProcess          1000f0e0 f i corelib0:cexit.obj
 0001:0000e0f8       _initterm                  1000f0f8 f   corelib0:crt0dat.obj
 0001:0000e14c       _cinit                     1000f14c f   corelib0:crt0dat.obj
 0001:0000e188       _onexit                    1000f188 f   corelib0:onexit.obj
 0001:0000e48c       atexit                     1000f48c f   corelib0:onexit.obj
 0001:0000e4e0       mbstowcs                   1000f4e0 f   corelib1:COREDLL.dll
 0001:0000e4f0       ??3@YAXPAX@Z               1000f4f0 f   corelib1:COREDLL.dll
 0001:0000e500       memset                     1000f500 f   corelib1:COREDLL.dll
 0001:0000e510       ??2@YAPAXI@Z               1000f510 f   corelib1:COREDLL.dll
 0001:0000e520       __rt_udiv                  1000f520 f   corelib1:COREDLL.dll
 0001:0000e530       memcpy                     1000f530 f   corelib1:COREDLL.dll
 0001:0000e540       _XcptFilter                1000f540 f   corelib1:COREDLL.dll
 0001:0000e550       __C_specific_handler       1000f550 f   corelib1:COREDLL.dll
 0001:0000e560       __security_gen_cookie2     1000f560 f   corelib1:COREDLL.dll
 0001:0000e570       __report_gsfailure         1000f570 f   corelib1:COREDLL.dll
 0001:0000e580       free                       1000f580 f   corelib1:COREDLL.dll
 0001:0000e590       malloc                     1000f590 f   corelib1:COREDLL.dll
 0001:0000e5a0       realloc                    1000f5a0 f   corelib1:COREDLL.dll
 0001:0000e5b0       _msize                     1000f5b0 f   corelib1:COREDLL.dll
 0001:0000e5c0       InterlockedExchange        1000f5c0 f   coredll:COREDLL.dll
 0001:0000e5d0       TerminateProcess           1000f5d0 f   coredll:COREDLL.dll
 0001:0000e5e0       InterlockedCompareExchange 1000f5e0 f   coredll:COREDLL.dll
 0001:0000e61c       __IMPORT_DESCRIPTOR_COREDLL 1000f61c     coredll:COREDLL.dll
 0001:0000e630       __IMPORT_DESCRIPTOR_CEDDK  1000f630     ceddk:CEDDK.dll
 0001:0000e644       __IMPORT_DESCRIPTOR_CSPDDK 1000f644     cspddk:CSPDDK.dll
 0001:0000e658       __NULL_IMPORT_DESCRIPTOR   1000f658     coredll:COREDLL.dll
 0002:00000000       __imp_MmUnmapIoSpace       10010000     ceddk:CEDDK.dll
 0002:00000004       __imp_MmMapIoSpace         10010004     ceddk:CEDDK.dll
 0002:00000008       \177CEDDK_NULL_THUNK_DATA  10010008     ceddk:CEDDK.dll
 0002:0000000c       __imp_GetLastError         1001000c     coredll:COREDLL.dll
 0002:00000010       __imp_SetLastError         10010010     coredll:COREDLL.dll
 0002:00000014       __imp_CeAllocAsynchronousBuffer 10010014     coredll:COREDLL.dll
 0002:00000018       __imp_CeOpenCallerBuffer   10010018     coredll:COREDLL.dll
 0002:0000001c       __imp_CeCloseCallerBuffer  1001001c     coredll:COREDLL.dll
 0002:00000020       __imp_CeFreeAsynchronousBuffer 10010020     coredll:COREDLL.dll
 0002:00000024       __imp_CeFreeDuplicateBuffer 10010024     coredll:COREDLL.dll
 0002:00000028       __imp_CeAllocDuplicateBuffer 10010028     coredll:COREDLL.dll
 0002:0000002c       __imp_CreateEventW         1001002c     coredll:COREDLL.dll
 0002:00000030       __imp_InitializeCriticalSection 10010030     coredll:COREDLL.dll
 0002:00000034       __imp_CloseHandle          10010034     coredll:COREDLL.dll
 0002:00000038       __imp_TerminateThread      10010038     coredll:COREDLL.dll
 0002:0000003c       __imp_WaitForSingleObject  1001003c     coredll:COREDLL.dll
 0002:00000040       __imp_DeleteCriticalSection 10010040     coredll:COREDLL.dll
 0002:00000044       __imp_NKDbgPrintfW         10010044     coredll:COREDLL.dll
 0002:00000048       __imp_InterruptDone        10010048     coredll:COREDLL.dll
 0002:0000004c       __imp_DevicePowerNotify    1001004c     coredll:COREDLL.dll
 0002:00000050       __imp_CeSetThreadPriority  10010050     coredll:COREDLL.dll
 0002:00000054       __imp_CreateThread         10010054     coredll:COREDLL.dll
 0002:00000058       __imp_InterruptInitialize  10010058     coredll:COREDLL.dll
 0002:0000005c       __imp_KernelIoControl      1001005c     coredll:COREDLL.dll
 0002:00000060       __imp_InterruptDisable     10010060     coredll:COREDLL.dll
 0002:00000064       __imp_LeaveCriticalSection 10010064     coredll:COREDLL.dll
 0002:00000068       __imp_EnterCriticalSection 10010068     coredll:COREDLL.dll
 0002:0000006c       __imp_RegCloseKey          1001006c     coredll:COREDLL.dll
 0002:00000070       __imp_wsprintfW            10010070     coredll:COREDLL.dll
 0002:00000074       __imp_RegQueryValueExW     10010074     coredll:COREDLL.dll
 0002:00000078       __imp_OpenDeviceKey        10010078     coredll:COREDLL.dll
 0002:0000007c       __imp_DisableThreadLibraryCalls 1001007c     coredll:COREDLL.dll
 0002:00000080       __imp_EventModify          10010080     coredll:COREDLL.dll
 0002:00000084       __imp_RegisterDbgZones     10010084     coredll:COREDLL.dll
 0002:00000088       __imp_TerminateProcess     10010088     coredll:COREDLL.dll
 0002:0000008c       __imp_InterlockedExchange  1001008c     coredll:COREDLL.dll
 0002:00000090       __imp__msize               10010090     corelib1:COREDLL.dll
 0002:00000094       __imp_realloc              10010094     corelib1:COREDLL.dll
 0002:00000098       __imp_malloc               10010098     corelib1:COREDLL.dll
 0002:0000009c       __imp_free                 1001009c     corelib1:COREDLL.dll
 0002:000000a0       __imp___report_gsfailure   100100a0     corelib1:COREDLL.dll
 0002:000000a4       __imp_mbstowcs             100100a4     corelib1:COREDLL.dll
 0002:000000a8       __imp_??3@YAXPAX@Z         100100a8     corelib1:COREDLL.dll
 0002:000000ac       __imp_memset               100100ac     corelib1:COREDLL.dll
 0002:000000b0       __imp_??2@YAPAXI@Z         100100b0     corelib1:COREDLL.dll
 0002:000000b4       __imp___rt_udiv            100100b4     corelib1:COREDLL.dll
 0002:000000b8       __imp_memcpy               100100b8     corelib1:COREDLL.dll
 0002:000000bc       __imp__XcptFilter          100100bc     corelib1:COREDLL.dll
 0002:000000c0       __imp___C_specific_handler 100100c0     corelib1:COREDLL.dll
 0002:000000c4       __imp___security_gen_cookie2 100100c4     corelib1:COREDLL.dll
 0002:000000c8       __imp_InterlockedCompareExchange 100100c8     coredll:COREDLL.dll
 0002:000000cc       \177COREDLL_NULL_THUNK_DATA 100100cc     coredll:COREDLL.dll
 0002:000000d0       __imp_DDKIomuxSetPadConfig 100100d0     cspddk:CSPDDK.dll
 0002:000000d4       __imp_DDKIomuxSelectInput  100100d4     cspddk:CSPDDK.dll
 0002:000000d8       __imp_DDKClockSetGatingMode 100100d8     cspddk:CSPDDK.dll
 0002:000000dc       __imp_DDKGpioSetConfig     100100dc     cspddk:CSPDDK.dll
 0002:000000e0       __imp_DDKGpioWriteDataPin  100100e0     cspddk:CSPDDK.dll
 0002:000000e4       __imp_DDKIomuxSetPinMux    100100e4     cspddk:CSPDDK.dll
 0002:000000e8       \177CSPDDK_NULL_THUNK_DATA 100100e8     cspddk:CSPDDK.dll
 0002:000000f0       dpCurSettings              100100f0     DebugZones.obj
 0002:00000534       __security_cookie          10010534     corelib0:seccinit.obj
 0002:00000538       __security_cookie_complement 10010538     corelib0:seccinit.obj
 0002:000014e4       _exitflag                  100114e4     corelib0:cexit.obj
 0002:000014e8       __onexitend                100114e8     <common>
 0002:000014ec       __onexitbegin              100114ec     <common>
 0002:000014f0       g_pcsExit                  100114f0     <common>
 0002:000014f4       _pRawDllMain               100114f4     <common>

 entry point at        0001:0000db4c

 Static symbols

 0001:0000dba0       _DllMainCRTStartupHelper   1000eba0 f   corelib0:pegdmain.obj
 0001:0000df28       doexit                     1000ef28 f   corelib0:cexit.obj
 0001:0000e1e4       lockexit                   1000f1e4 f   corelib0:onexit.obj
 0001:0000e280       unlockexit                 1000f280 f   corelib0:onexit.obj
 0001:0000e2ac       _onexit_nolock             1000f2ac f   corelib0:onexit.obj
